:1020000000800020755C00005D5C00005D5C0000ED
:1020100000000000000000000000000000000000C0
:102020000000000000000000000000005D5C0000F7
:1020300000000000000000005D5C0000C95C0000C2
:102040005D5C00005D5C00005D5C00005D5C0000AC
:10205000215C00005D5C00005D5C0000615C0000D4
:102060005D5C00005D5C00005D5C00005D5C00008C
:102070005D5C00005D5C0000ED5900005D5C0000EF
:102080005D5C00005D5C00005D5C0000C527000039
:10209000000000005D5C00005D5C00005D5C000015
:1020A0005D5C00005D5C00005D5C00005D5C00004C
:1020B0000000000010B5064C2378002B07D1054B1B
:1020C000002B02D0044800E000BF0123237010BDA4
:1020D000A00200200000000058E60000044B10B5EC
:1020E000002B03D00349044800E000BF10BDC046E8
:1020F00000000000A402002058E60000002370B594
:102100000E4C23602168B42908DC0D4800F05AFC0D
:102110000F2003F01DFE23680133F2E7094D0A4941
:10212000280005F0D7FF0A222168280006F03BF8B6
:102130002800064905F0CEFF70BDC046C40200204D
:10214000BC020020BC0900206DDB0000EDE10000B6
:10215000B42370B50E4C23602168002908DB0D48BC
:1021600000F030FC0F2003F0F3FD2368013BF2E7A1
:10217000094D0A49280005F0ADFF0A222168280010
:1021800006F011F82800064905F0A4FF70BDC0460E
:10219000C4020020BC020020BC09002010DB0000AB
:1021A000EDE1000010B5024800F0D4FE10BDC046BD
:1021B0006003002070B5154C1549200005F08AFF1A
:1021C000144D2000290005F085FF1349200005F07B
:1021D00081FF124A2900124800F0E8FC032807D0CA
:1021E0001049200005F076FF0F4803F0B1FDF0E73D
:1021F000200005F079FF0D49200005F087FFFFF76B
:10220000D1FF200005F070FF70BDC046BC09002062
:102210002BDB000090DB000020E6000087DB0000E5
:10222000600300204BDB0000881300004DDB000042
:10223000F0B5694895B000F031FD032801D0FFF7F3
:10224000B9FF664B1868C0B203F00EFF644D2860FA
:1022500008F080F80022634B07F070FA0022624B0E
:1022600007F06CFA0B000221020000910EA806F0A4
:1022700065F80EA911A806F04CF85C4911A806F003
:10228000BDF85B4C0100200005F036FF11A805F0F9
:102290009EFF0EA805F09BFFFA20400003F058FDBA
:1022A000544905A805F0E2FF00F0CEF90A2201002A
:1022B00002A805F0FAFF02A905A806F092F84E4917
:1022C00006F09CF8060000F0C9F90A22010008A8EF
:1022D00005F0EBFF08A9300006F083F8474906F047
:1022E0008DF8060000F0C4F90A2201000BA805F0E1
:1022F000DCFF0BA9300006F074F8414E310006F007
:102300007DF8070000F0BEF90A2201000EA805F0D2
:10231000CCFF0EA9380006F064F8310006F06EF824
:10232000060000F0B9F90A22010011A805F0BDFF6E
:1023300011A9300006F055F80100200005F0DCFE80
:1023400011A805F044FF0EA805F041FF0BA805F009
:102350003EFF08A805F03BFF02A805F038FF05A8DE
:1023600005F035FF274911A805F080FFFFF71AFF98
:102370000A2201000EA805F0AAFF0EA911A806F076
:1023800030F80100200005F0B7FE0EA805F01FFF91
:1023900011A805F01CFFFFF705FF002804D0FFF788
:1023A00001FF002100F0F8F8286807F0D3FF0022B1
:1023B0000C4B07F0C3F90022134B06F071FA00280A
:1023C00007D0FFF79BFEFA20C00003F0C1FC15B058
:1023D000F0BDFFF7BDFEF6E760030020040000201B
:1023E000C00200200000503F0000594098DB000070
:1023F000BC0900209ADB0000B4DB000020E60000EE
:10240000B6DB0000B8DB00000000E03F10B5034879
:1024100000F0ACFE024800F0DFF910BDC802002059
:10242000BC02002010B50921044800F09BFA962157
:102430000348890104F074F910BDC046BC020020B5
:10244000BC090020F7B53C211500040006F022F974
:10245000200029703C2106F097F83C2106F01AF97B
:102460006970E1212000090106F08EF8182106F0BC
:1024700011F92000A970344906F086F80024019073
:102480000721043006F006F926000131E9702F4BD0
:10249000F71803233B40009317D16421380006F05E
:1024A000E3F9B7235B00002908D19131FF313800EF
:1024B00006F0DAF94B424B416E33FF33E418019BCF
:1024C000A34204D30136F6B2E1E76E23F5E7AE711D
:1024D0006421380006F0C8F90E00C8213800490010
:1024E00006F0C2F9009B002B25D1002E25D14B42CE
:1024F0004B416E33FF331D22E41A019B94464A423E
:1025000051411C1B00231C31D8B2012B18D1009F54
:102510001C22002F03D16246002E00D10A00A242E5
:1025200004D80133A41A0C2BEED118000130013469
:1025300068712C71F7BD6E23DCE7B7235B00DAE727
:10254000034A9A5CEBE7C04680510100B2070000E5
:10255000D3DB000070B5084C060023680D008342F1
:1025600002D163688B4206D0044A30002900FFF78D
:1025700069FF2660656070BDF0020020E402002063
:1025800010B5FFF7E7FF024B9879024BC01810BD5A
:10259000E4020020B20700000222074B10B51860C9
:1025A000064B1B681818064B1860064B1A7003F090
:1025B00099FB054B186010BDEC02002008000020BC
:1025C000E0020020EB020020DC02002070B503F0E6
:1025D00089FB1649164A0B68164CC01A904207D957
:1025E000226801322260FA2292009B180B60EEE70B
:1025F000114D22682B68934209D8104B1B68002BA1
:1026000005D0984703000B4304D0FFF7C5FF2068AF
:10261000002170BD0A4B22681B68D318094A2B6041
:102620001378591E8B411370F1E7C046DC0200207D
:10263000E7030000EC020020E0020020F802002086
:1026400008000020EB02002010B5FFF7BFFFFFF7E6
:1026500081FF014B987810BDE402002010B5FFF710
:10266000B5FFFFF777FF014B587810BDE40200205B
:1026700010B5FFF7ABFFFFF76DFF014B187910BDE9
:10268000E402002010B5FFF7A1FFFFF763FF014B45
:10269000587910BDE402002010B5FFF797FFFFF74F
:1026A0006FFF10BDF7B50C27404E0193335C04005B
:1026B0005BB20D0000924743002B2EDA00230B8201
:1026C000EB7BDB09FCD1335D394A01335BB2335517
:1026D000335D12785BB2DB19934203DA335D5BB290
:1026E0000B2B34DD2F8ABFB2EB7BDB09FCD1314BE6
:1026F0003149186805F048FF304B04375843009BB8
:1027000000090C3387424DD280B25B005853EB7BFB
:10271000DB09FCD1FF33335540E0335C244A5BB224
:102720001278DB199342CEDA335C254A5BB2DB19AF
:10273000DB009B5C5B06C6D5335C00215BB2DB191A
:10274000DB00985C8006800E03F048FDBBE7335D3C
:102750001B4A5BB2DB19DB009B5C5B0609D5335D72
:1027600001215BB2DB19DB00985C8006800E03F070
:1027700035FD2A8A92B2EB7BDB09FCD1335D5BB27B
:10278000DF190F4BFF00DF197B68D318009A9BB24B
:102790000C3252005353EB7BDB09FCD16B461B79A7
:1027A000AB73F7BDBFB25B005F53B0E7FD02002023
:1027B000FC0200201400002040420F00204E0000C8
:1027C00000030020002210B5102302491000FFF77B
:1027D00069FF10BD0030004270B50C4B05001C783D
:1027E0000B2C10D8621C1A70094B04701868094928
:1027F00005F0CAFE084BE4005843084B00091C19B9
:102800006060280070BDFF230370FAE7FC0200201F
:102810001400002040420F00DC05000000030020EF
:10282000F7B50193037804000E0017000B2B00D9B5
:1028300086E0C8B2012103F085FC3F2132002078F8
:10284000404DC3005E5D0A408E4316435E558823AB
:10285000032296219B00DB1BDF171740FF18019B0B
:102860000901C91ACB1713405B189B10BF10A37046
:1028700067700C2105F088FE0C23C0B243431A0098
:102880000C32D900695C490654D401339342F8D123
:1028900000284FD12C4B2D4A5A805A78D209FCD1AE
:1028A0002B4E0232338893433380F37BDB09FCD118
:1028B00001333380F37BDB09FCD13388DB07FCD4A5
:1028C00033889BB233804023328813433380802384
:1028D0003288DB0013433380012332791343337191
:1028E000F37BDB09FCD11B4B1B49186805F04CFE40
:1028F0000300FA2080005843000980B23083F37B44
:10290000DB09FCD18021154B0903D967C023C42002
:10291000134A5B00D150800013581B021B0A13504E
:1029200010231160737332880E3B13433380F37BA3
:10293000DB09FCD140222378DB00E95C0A43EA543E
:102940002078FEBD00030020000C00401C40000069
:10295000003000421400002040420F0004E100E07B
:1029600000E100E09623882210B51B019200FFF7DA
:1029700057FF10BD70B505780B2D1BD80123882497
:10298000C356E41AA4008C4208DC96248078A40084
:1029900040B2241AA4008C4200DD0C00064B07490B
:1029A000186805F0F1FD053C6043054BED0000099A
:1029B0005D19686070BDC0461400002040420F00E1
:1029C000000300200F4B13B50400994216DCB4201D
:1029D000B42902DCC843C017084001228823A2564C
:1029E00002219B1A962261569200521A920000927E
:1029F00000219B00B42205F02BFA01002000FFF714
:102A0000B9FF13BD1F020000014B19627047C04699
:102A10006003002010B502F055FE10BD30B587B040
:102A2000040000F069FC134B6846009301F0A2F823
:102A3000051E02D003000D3319D102F035F90E49FD
:102A40000E4802F04DF921000023012229312260B5
:102A50000B70E2610A4A23616361A36123626362CE
:102A60001268084B9A4202D9D32000F069FF28006F
:102A700007B030BDE12E0000092A0000152A000031
:102A8000F00300204F130000F8B503680400002B8A
:102A900001D1FFF7C3FFE369002B03D000232361BB
:102AA0006361A361250001F0A1F82935002802DA4D
:102AB00004202870F8BD002326002B70283601332F
:102AC000337003F00FF9070003F00CF9236FC01BFC
:102AD000984206D2002001F085F807222B78134295
:102AE000F2D0200021224D30002107F043FD0322C7
:102AF0002B78134002D133702878DBE701F06CF9B2
:102B0000002001F06FF8F7E7F0B51F00036885B00B
:102B100004000D001600002B01D1FFF77FFFE369D1
:102B2000002B03D0002323616361A361280008F018
:102B300003FDFF23C1B2009332003B0028002600B2
:102B400001F0EBF82936002805DA042333701E0063
:102B5000300005B0F0BD0023270033702837013363
:102B60003B7003F0BFF8039003F0BCF8039BC01A5E
:102B7000236F984206D2002001F034F80722337800
:102B80001342F1D003233678334000D13B704D34EB
:102B900021220021200007F0EDFC280008F0CCFCE9
:102BA00029000200200007F0C9FCD1E710B513008E
:102BB0000222FFF7A9FF10BDF0B51F000368A5B002
:102BC00004000D001600002B01D1FFF727FF88221B
:102BD000002102A807F0CEFC290002A808F0A4FCFE
:102BE00002AB0233DF773F230122002702A95B18E3
:102BF0001A70412012AB1F70C02309180B7002A974
:102C00007E3B5B18A8211970432302A95B181A7038
:102C1000310013AB02A81A70260001F095F829368E
:102C2000B84203DA0B20307025B0F0BD0A233370B0
:102C30002300022228331A70253318001F3239006E
:102C4000019307F097FC280008F076FC29000200A9
:102C5000019807F073FC4123200002A95B18103093
:102C60001900042200F012FC024B63612369A36186
:102C70003078D9E7FFFFFF0037B56D4608000C003C
:102C800001F054F8280001F051F80023EA1A5279B3
:102C9000E2540133062BF9D120003EBD10B5036884
:102CA0000400002B01D1FFF7B9FE2934002000F009
:102CB00099FF207810BD000030B587B004000D00EA
:102CC000FFF7E2FE032811D069462000FFF7D4FF8A
:102CD0006B466A461B785278074902A808F0FAFB4F
:102CE0002B00064A02A92000FFF766FF2000FFF72D
:102CF000D5FF07B030BDC046DFDB0000F0DB0000D1
:102D000010B50121FFF7D8FF10BD0000F0B5040099
:102D100085B01500132900D1A1E011D8062900D1F2
:102D2000C8E003D8042965D005B0F0BD092965D0F5
:102D30001129F9D11378002BF6D02934022325E08C
:102D40002A291DD00AD81B29EED1006A0028EBD011
:102D50000822290007F0F2FB00234DE02C2917D0B0
:102D60003229E1D1030028331B78012BDCD1136811
:102D700029340361D368436153688361032305E009
:102D80000023D356002BCFD0062329342370CBE762
:102D90001378012B0FD1030028331B78012B05D1A9
:102DA000C369002BC0D129340333EFE7032BBBD118
:102DB00029340533EAE7002BB6D102002832127815
:102DC000012A12D10200062129321170C269002A9B
:102DD00002D0036143618361002461B23F48013442
:102DE00002F0F4FA0B2CF8D19EE7032A9CD1293487
:102DF0000723CBE70023D356236295E71300633301
:102E00001E78002E24D107004D37310021223800D2
:102E100007F0B0FB280008F08FFB29000200380003
:102E200007F08CFB2300012228331A70280026614A
:102E30006661A66108F080FB2A002B00C1B2FF206A
:102E40006232127821330090280000F066FF6BE7B1
:102E500003000B2229331A70FFF752FF64E71300B7
:102E60000A331800039308F067FB270006002A378F
:102E700021220021380007F07DFBB3B2002B04D0E3
:102E80001A000399380007F059FB636A002B07D03A
:102E90000023EA1A527A616ACA540133062BF8D128
:102EA0000123EB5623622300AA784B331A70EA7889
:102EB0005A7042E7436A002B0AD000232B32117864
:102EC000606A013AC1540133062BF8D100236362D2
:102ED000200029004D3008F027FB25E7FC030020E7
:102EE00010B50A0001000248FFF710FF10BDC046F0
:102EF00060030020F8B5040010000E00150004F077
:102F0000F3FF0123002806D12062300002F07AF896
:102F1000002802DA00231800F8BD02F0E3FE0700E3
:102F2000266A002E09D102F0DDFE094BC01B984233
:102F300003D8300000F056FEF2E7216A0029E9D0FC
:102F4000280005F004F8002323620133E3E7C046BC
:102F50001F4E000070B58CB001AC0462050000F09B
:102F600047FF02F0BFFE06002B6A002B09D002F0DB
:102F7000B9FE134B801B984203D8002000F032FEAC
:102F8000F2E700202B6A834216D12388834213D0B4
:102F90000C4A03A89B180893A378013B0793E37896
:102FA00006932379059363790493A379039301230B
:102FB0005B420B9307F0B0FB00232B620CB070BD9B
:102FC0008713000094F8FFFF064B002219002831F8
:102FD0000A701A601A00FF2129321170024A1A671A
:102FE0007047C0466003002060EA00000020704780
:102FF00013B56B460268D971073354681900012272
:10300000A04716BD13B56B46DC1D036801225B6A41
:1030100021009847012801D1207816BD01204042A7
:10302000FBE77047007C40B20130431E9841C0B2BC
:1030300070470000102110B541560400002904DB40
:10304000024802F0C3F9FF23237410BDFC030020E3
:10305000102110B5415600204B1C02D0014802F04F
:103060006EF910BDFC030020036870B51B690400F5
:103070000D001600984780B2002807D010213300B9
:1030800061562A00034802F03CFA70BD012040421C
:10309000FBE7C046FC030020036810B51B69040071
:1030A0009847002805D010210348615602F0FEF928
:1030B00010BD01204042FBE7FC030020102110B5A9
:1030C00041560020814202DB014802F029F910BD7F
:1030D000FC030020102213B58A560400531C07D1AC
:1030E000002100910B000A0004F0E8FE200016BD4C
:1030F000014902F038F9F9E7FC030020102170B50E
:103100004156060000204B1C0DD0074D280002F050
:1031100034F9102104007156280002F02EF924021F
:103120000012204380B270BDFC03002070B5037C08
:1031300004000E0015007F2B06D8002A04D0036877
:10314000DB6A9847002804D101230025636028002A
:1031500070BD10212B0061563200034802F012F9B5
:103160000028F4DCF0E7C046FC03002000234360A5
:10317000FA239B008360034B08330360FF2303742F
:103180007047C046F8DB0000F0B589B00393022316
:1031900004AE33804B6852BA736003687280DB6A96
:1031A00004009847002803D0236820009B6A9847B2
:1031B000194D039B01220221280002F059F8070053
:1031C00020740020874224DB039BDB070ED50E9B77
:1031D00083420BD0180000F06BF90E9B0190009316
:1031E000022339001A00280002F053F8102132009F
:1031F00061561023280002F057F806000120002E27
:1032000007D110212800615602F0E0F8FF233000BA
:10321000237409B0F0BDC046FC0300207FB5064B07
:1032200004934B6804A90393059300230093FFF7CD
:10323000ABFF07B000BDC046E8E10000F0B50C00F0
:1032400089B0050004A816001F0004F02FFE04AA90
:1032500021000948FFF74EFE00280BD0074B0094D1
:103260000693059B32000393079306A93B002800B1
:10327000FFF78AFF09B0F0BD60030020E8E100001D
:1032800010B50023FFF7DAFF10BD0000034B10B5A7
:103290001B68002B00D0984710BDC046D403002007
:1032A00010B5D2B2C0B202F0E9FB10BD10B5C0B289
:1032B00002F07CFC10BD10B50400013C00D210BD32
:1032C000012002F045FDF8E7002010B5094C20561A
:1032D00000280DDB0021C0B202F080FF6420FFF760
:1032E000EAFF2078012102F079FF6420FFF7E3FF75
:1032F00010BDC0460F0000200022002010B5104B6A
:10330000104C1A602056904207DBC0B2012102F037
:1033100019FF2078012102F061FF0B4B0021187882
:1033200002F010FF0020094B1856002803DBC0B242
:10333000022102F007FFFFF7C7FF002010BDC046C3
:10334000D40300200F0000200E0000200C000020FD
:10335000054B10B518600020044B03221856044991
:10336000FFF79EFF10BDC046D40300200E000020D2
:103370008D3200000300002010B5064A1056002BC5
:1033800004D003220449FFF78BFF10BDFFF78EFF27
:10339000FBE7C0460E0000208D320000034B044ABC
:1033A0001A6000221A7101325A717047D803002046
:1033B000001BB70010B5094802F088FA084C01213B
:1033C000207802F0BFFE2078012102F007FFFFF70E
:1033D0007BFF0120FFF76FFF002010BD8806002053
:1033E0000D000020F0B585B003283ED1002202ABCD
:1033F0000D6807330C894E681A70954222D09642A8
:1034000030D101961E0001320092194B194F06CBA4
:10341000380002F083FA184B0021187802F0DEFE23
:10342000002C14D02978380002F081F9009B30700C
:103430005A425341F618019B013C5A425341A4B2EF
:10344000ED18EDE70122009501921D00DDE70A4B22
:103450000121187802F0C2FE380002F0DFF92000E6
:1034600005B0F0BD06204042FAE70120FBE7C04668
:10347000D8030020880600200D00002010B5024867
:1034800002F04DF9002010BD8806002010B5002A7A
:1034900005D00023CC5CC45401339A42FAD110BD4C
:1034A000002A04D08218017001308242FBD170479B
:1034B0000023C15C9AB201330029FAD11000704791
:1034C000024AD3780133DBB2D3707047201000205A
:1034D00070470000002307B50A4A012013700A4A0A
:1034E0009370FFF747FF01A9084800F07FFE00280E
:1034F00006D10221019B05481943019100F07AFE93
:103500000EBDC046E0030020201000207010000017
:10351000002010B50A4CA378834207D16378834218
:1035200005D0002063780133DBB2637010BD2378CF
:10353000002BF6D000F024FD0028F2D0F6E7C046BC
:1035400020100020044A5378002B03D05378013B0D
:10355000DBB25370002070472010002010B5094BDB
:103560005A78002A03D05A78013AD2B25A70002011
:103570005A78824204D11B78834201D000F0D2FCF9
:1035800010BDC0462010002010B5064C2822002196
:103590002000FFF785FF0448FFF7DAFE034B002009
:1035A000E36110BD20100020C1340000D1340000C0
:1035B000F0B58DB0019312AB049204CB07000292D8
:1035C0007F221B880A40039314AB1B880D000593D0
:1035D00008AB5A70082218705A80029A002A45D007
:1035E00003995A8852180599521892B25A80FFF7D7
:1035F0008FFF041E37D106AB0A90D88009909E1D1C
:10360000099B2D021F430997099B49481D430995B2
:1036100008AD6B88099A1B0413430993099900F0BC
:10362000E9FD041E38D102270990099B41483B431C
:103630000993099900F0DEFD041E2DD10A90308017
:1036400006AB9C1D22883C4B9A4205D809A93948F3
:1036500000F0CCFD00280CD00A9B002B26D10324BF
:10366000FFF77CFF644220000DB0F0BD5A8801993D
:10367000BAE7F4232288FF339A4203D90120238832
:10368000FFF719FE099E3E4009D10AA92B4800F018
:10369000ADFD041EE0D00A96FFF754FFE3E706AB4A
:1036A0009A1DDB8801339BB21380C9E70A9B08226D
:1036B0000B936B8829009BB26B800B9800F0BCFDCC
:1036C000041EE9D10B9B08330B93049B002B0AD0FB
:1036D0000B98019A190000F0AFFD041EDCD10B9B82
:1036E000019AD3180B93029B002B10D00199059BD4
:1036F0000B9A5B1A9B180B930B98039A029900F094
:103700009BFD041EC8D10B9B039AD3180B930A9BF5
:103710000B489B0009930223099A134309930999C3
:1037200000F068FD041EB7D1FFF718FF04009AE708
:103730008C10000078100000E70300000004150062
:103740006C100000F0B5544B87B01B78002B32D0C2
:1037500000230193019807B0F0BD63889F4209D010
:103760006388FF1A042F05DD0120FFF703FE0626FC
:10377000764261E02378012B60D1EB68002B08D002
:10378000EB6860786188059A0839C0B2083289B25E
:103790009847414B1B78002B06D1AB78002B03D008
:1037A000FFF798FE061E47D13B4B1B78002BD1D16B
:1037B000019B002B07D1394DEB78002BC8D0EB785B
:1037C000013BDBB2EB7003A9354800F00FFD01901F
:1037D0000028E9D10122039B1342E5D00124FFF721
:1037E000C9FD039B2E48A3430393039900F002FDF8
:1037F00001900028D8D1AC70039FBF043F0D46D084
:10380000059005A9274800F0F1FC06002000002ED5
:1038100010D1059B04AC1800042221006B60AF603E
:1038200000F0ECFC0190638806009BB263800028E6
:1038300093D00120FFF79EFD0196B5E72378022B78
:1038400004D12B69002BA4D02B699AE72378042B91
:1038500004D16B69002B9CD06B6992E72378062B0F
:1038600004D12B6A002B94D02B6A8AE72378072B8C
:1038700004D1AB69002B8CD0AB6982E72378052B90
:1038800000D074E76B6A002B83D06B6A79E7022360
:103890005B42019388E7C046E0030020201000202F
:1038A0007010000084100000F8B51D00002803D03F
:1038B000002901D0002A04D1002D1BD0FFF70AFEF9
:1038C00017E00E4CA3689A4214D86368834211D85B
:1038D0006368A7681618DB199E420BD800F08EFCAF
:1038E000002806D16368A2689B189E42E6D0002D8E
:1038F000E4D1F8BD0C204042FBE7C0462010002078
:10390000013800B5062815D80C4B04F033FE070427
:103910000B09110D0F001961002000BDD960FBE7F4
:103920005961F9E7D961F7E71962F5E79961F3E7BA
:103930005962F1E70C204042EFE7C046201000201A
:103940007FB500230521059002930193009305AAFA
:1039500004330800FFF72CFE07B000BD70B504006B
:103960009AB015002C2802D10023042203E01B2862
:103970000ED10023082201A92800FFF795FF002897
:1039800004D1524B01A91B68002B38D11AB070BD6D
:10399000062802D101233022EDE70E28F6D0322886
:1039A00015D14B4A4B4B11681422994200D8043A66
:1039B000002301A92800FFF777FF0028E6D1434B39
:1039C0001B68002BE2D001A932309847DEE72F2890
:1039D00007D16422002101A8FFF762FD00236422C1
:1039E000C9E734280DD101A9002304222800FFF7DC
:1039F0005BFF011ECAD1354B1B68002BC6D02000CF
:103A0000E3E7112814D10023334A01AC13702100DD
:103A100004222800FFF748FF0028B7D12F4B227857
:103A20001A702A4B1B68002BB0D021001130CCE754
:103A300013280ED100232C2201A92800FFF734FF00
:103A40000028A3D1214B1B68002B9FD001A9133064
:103A5000BBE7042810D10023042201A92800FFF7A6
:103A600023FF002800D091E7184B1B68002B00D1E2
:103A70008CE701A90430A8E7652800D174E709287C
:103A800001D10123ABE72A2801D101236DE72028CA
:103A900000D07BE701AE0023082231002800FFF7A9
:103AA00003FF002800D071E72800B2880830012306
:103AB0000199FFF7F9FE002800D067E7034B1B6868
:103AC000002B00D162E7310099E7C046E4030020F3
:103AD000F00300204F130000E9030020E80300205A
:103AE00010B5041E3BD0FFF7E3FC002837D02000C0
:103AF000FFF7DEFC202832D8A31CDB7F013B0D2B17
:103B00002DD8230041331B78002B09D123004233E9
:103B10001B78002B04D1230043331B78002B1ED0CD
:103B200023003F331B78012B01D1002010BD032B54
:103B300018D1E31CDB7F013B032B10D81022231D7F
:103B4000DB7F93430A2B0AD124342000FFF7B0FC1B
:103B5000002804D02000FFF7ABFC1A28E5D90C2080
:103B60004042E3E7022BFAD10434E37F083B382BD1
:103B7000DBD9F4E770B58CB06B46012607331E70B5
:103B8000002826D000250168134A18001160134A46
:103B9000157000F027FC0400A84213D1FFF7F4FCD5
:103BA0000400A84211D10E493000FFF7A9FE02A877
:103BB00000F0B8FB030004000C3303D102A800F0AE
:103BC00059FB040020000CB070BD280000F043FC3D
:103BD000F8E70C246442F5E7E4030020E903002041
:103BE0005D39000010B5FFF7ADFD10BD1FB5002217
:103BF000292102920192009213000120FFF7D8FCC4
:103C000005B000BDF0B5A5B01C002AAB1B8806901E
:103C100005932BAB1B780F0016000793012A1DD0CC
:103C2000002C03D10C20404225B0F0BD022A15D152
:103C30002000FFF73DFC402810D121002200403138
:103C40001378180030383628ECD80A380628E9D915
:103C5000473B192BE6D901328A42F1D17B1E1F2B3B
:103C6000E0D8059B013B0D2B02D9059BFF2BD9D139
:103C70005A2004AB09AD3A000699C018EF19FFF7B6
:103C800005FC3B00002746331F701A2304AA9B182B
:103C90006A46928A04A9DA87079B5A1E93417B22BF
:103CA0005218137055235B181E70032E1ED12378F3
:103CB0002B70032BB6D86278102311006A709943D9
:103CC0000A29AFD1162004ABC018A11CFFF7DEFBF8
:103CD0006378EB189F7000232A00029301930093EE
:103CE00028216C330120FFF763FC9DE7022E0DD1E4
:103CF0002000FFF7DDFB431E9BB2421C3F2B00D987
:103D000090E721002800FFF7C1FBE4E7042E01D172
:103D10003E22F6E7012EDED084E737B5002506AC5B
:103D2000248801950094FFF76DFF3EBD10B5040097
:103D3000FFF7EEFB002806D1200000F00DFA002866
:103D400001D1FFF70BFC10BDF0B50500B9B00C00B8
:103D50001600002836D0FFF7C3FE071E32D105A893
:103D600088222900FFF792FB2000FFF7A1FB002823
:103D700028D0002C26D027AD402221002800FFF7B4
:103D800085FB37AB1E70114B114A1F70114B196820
:103D9000CC2391420BD816226A44D37F2100013BE9
:103DA000D37717A84022FFF771FB8A232E700022D9
:103DB0008821029201920092012005AAFFF7F8FBE8
:103DC00039B0F0BD0C204042FAE7C046E9030020BC
:103DD0004F130000F00300201FB5002205210292BE
:103DE0000192009213000120FFF7E2FB05B000BD35
:103DF0001FB500221A2102920192009213000120A5
:103E0000FFF7D6FB05B000BD37B58024A5256400BB
:103E100004436D012100280000F0ECF9002301A902
:103E20002800019300F0E2F90028F3D1019BA3429E
:103E3000F0D13EBD002307B5104801A9019300F061
:103E4000D5F9002819D18021019B490019430B485D
:103E5000019100F0CFF900280FD1D02001A9400135
:103E600000F0C4F9002808D18021D020019B49022C
:103E700019434001019100F0BDF90EBD0814000086
:103E800037B51F4C2568002D20D18020210040012E
:103E900000F0ACF9002803D00023236028003EBDC9
:103EA00001A9184800F0A2F90028F5D12368164AA4
:103EB00093420DD1019B012B01D0144B2360236849
:103EC000134A1A40A023DB02134323602568E5E769
:103ED000104A934208D1019B032BF0D0042B01D14F
:103EE0000D4BEBE70D4BE9E70D4A9342E7D1EC2090
:103EF0002100800300F07AF90028CDD1DFE7C04629
:103F0000EC030020F4130000A0021000A102100036
:103F1000FFFFF0FFB0021000B1021000B20210006B
:103F2000F000100013B5012401A9102000F05EF983
:103F3000002812D1019B2342F6D101A9013000F0E3
:103F400055F9002809D102230199194206D101A986
:103F50000B2000F04BF9002808D016BD9943012032
:103F6000019100F047F90028F1D0F6E7012301990B
:103F70001942F2D099430B20019100F03BF9ECE794
:103F8000002373B50B2069460093019300F02EF9CE
:103F9000041E09D10121009B0B4207D06946012074
:103FA00000F024F9041E08D0200076BD19430B2030
:103FB00000F020F9041EF1D0F6E70221009B0B422D
:103FC00013D00525042601A90F2000F00FF9041EC7
:103FD000EAD1019B33420FD10220013DFFF76BF97B
:103FE000002DF0D104246442DEE71943012000F0E3
:103FF00001F9041EE5D0D7E700F0F0F8D4E700009F
:1040000070B50400264800F0EDF8002803DB01201D
:10401000FFF751F9F6E7234800F0E4F8C3070CD4A2
:10402000214D0120FFF747F9013D204800F0DAF863
:10403000002D31D01E4B9842F3D1022C0AD11D49DC
:104040001D4800F0D7F8802149031C4800F0D2F841
:1040500000240EE0032C05D11649174800F0CAF8D9
:104060000021F2E716491548042CEFD100F0C2F800
:104070007C34FFF705FF134B0005000D984209D96A
:1040800002202043FFF7C0FE0F49084800F0B2F8B5
:10409000002070BD2000F5E705204042F9E7C0464A
:1040A00014100000BC070200D10700000C000C0037
:1040B0009ED0AD107DD51C3CAC0702008C100000DA
:1040C000521352139F030000612F52EF37B5134B69
:1040D000134C023800930194012803D8114B00932C
:1040E000114B0193FA250020ED00019B834209D179
:1040F000019B0025A34203D12900084800F07AF86B
:1041000028003EBD0220FFF7D6F8013D009800F0E0
:1041100069F8002DE9D105256D42F1E78C1000000A
:1041200036265302AC070200C3C15DD707B5A020F5
:10413000002301A94001019300F058F8002807D19D
:10414000A020019B034940011940019100F052F861
:104150000EBDC046FFFBFFFF30B587B0082200212F
:10416000050004A806F006FA01A9164800F03EF87A
:10417000041E24D1019B002B1BD0C02080021843B9
:10418000082204A900F03AF8041E18D1049B0193F8
:10419000019B02A998B2C0239B02019006221843FA
:1041A00000F02CF80622040002A92800FFF76EF99F
:1041B00005E001A9044800F019F8041EE8D0200029
:1041C00007B030BD08000C009C14000010B5FFF7CC
:1041D000F1F810BD10B5FFF751F910BD10B500F0A2
:1041E000DFFA10BD10B500F0EFFA10BD10B500F009
:1041F000F1FA10BD10B500F0F6FA10BDF7B50700E2
:10420000150006000B4B01911C88083CA4B2019BD1
:10421000D91B8919AC4204D3AAB2300000F02CFBA0
:10422000FEBD2200300000F027FB0028F8D12D1B36
:104230003619ECE710000020F7B50700150006005E
:104240000B4B01911C88083CA4B2019BD91B891916
:10425000AC4204D3AAB2300000F056FBFEBD2200EF
:10426000300000F051FB0028F8D12D1B3619ECE787
:1042700010000020002373B5040001A92348019316
:10428000FFF7B4FF224B019A05009A4204D101A91D
:104290002048FFF7ABFF05000F26019A110C8BB2E7
:1042A000180A1B0933402372314093B26172190A14
:1042B0001B093340324021716371A271E071FFF735
:1042C000DFFD00232060FF2022792384A3791202DE
:1042D0003340134362791201024013430E4A1360C4
:1042E000E179627A090232400A43217A09010140E8
:1042F0000A480A43824201D90D256D42084A934279
:1043000001D80D256D42280076BDC046AC070200DD
:10431000C3C15DD748100000F00300205213000015
:104320005113000030B5002585B004000822290093
:1043300002A8019506F01EF9AC4202D1002005B09A
:1043400030BD290020002822FFF7AAF801A9214842
:10435000FFF74CFF0028F2D10198002802D10C2071
:104360004042ECE7C025AD022843082202A9FFF72E
:1043700045FF0028E3D1039880B201900028EED0D9
:10438000284328222100FFF739FF0028D7D10F2129
:10439000FF252279A379607912020B4000011343B3
:1043A00028400D4A03431360627AE0790A40217A7B
:1043B00000020901024329400A43002BCFD0002A02
:1043C000CDD006498A4202D8054A9342B6D80D207C
:1043D000C6E7C04608000C00F0030020521300009E
:1043E0005113000070B50125002804D005786B1E1C
:1043F000032B00D901250020FFF7E8FE041E1ED183
:10440000FF24FFF73DFDE823240120409B00984254
:1044100017D100F0F1F92800FFF7F2FD041E0CD1CE
:104420002800FFF753FE041E07D1023D012D06D9D7
:10443000FFF700FD002802D00400FFF7CBFE2000AC
:1044400070BDFFF71DFDAC2320409B009842E0D0DB
:1044500010246442F1E710B5FFF768FE041E09D18D
:1044600000F074FE041E05D1FFF7B4FE041E01D156
:1044700000F0A4F9200010BD1FB5002201AB01908F
:104480001981032019000292FEF7ACFF05B000BDB0
:104490001FB5002201AB029019810320190001927F
:1044A000FEF7A0FF05B000BD73B56B460600DD1D2D
:1044B000CF2822D003003B33DBB2012B1DD90B24C4
:1044C00001212800FFF7E4FF00281CD12B78B3421C
:1044D00003D0013CE4B2002CF2D10B2401212800CE
:1044E000FFF7D6FF00280ED12B78002B03D0013C1C
:1044F000E4B2002CF2D1012006E001212800FFF7F0
:10450000C7FF0028DBD0002076BD0000F0B50C000E
:10451000002785B0009001928023261C9B019C42BD
:1045200001D91B4B1E880A25B6B202AB0121D81C4B
:10453000FFF7AEFF002808D102ABDB781B090F2B79
:1045400010D0013D2DB26B1CEFD100201DE0114BAE
:104550001B78002B12D1022103A8FFF799FF002836
:104560000CD0F2E7002DF0D0009B3100D819FFF7F6
:104570008FFF0028E9D1019B002BE8D0A41BF7197D
:10458000A4B23FB2002CC7D1012005B0F0BDC04697
:104590003CDC0000F4030020F0B585B00AAC2578BF
:1045A00001AC2070C3380C2800D96BE003F0E2FFA7
:1045B000482936363C3C5A076A6A6A6A3A000B0C4C
:1045C00063700B0AA370E17005212F4B481E1B7806
:1045D000002B55D10A002D4D7F3366185742F75DE9
:1045E0005B007B40013AEB5C012AF7D15B0023546E
:1045F00089B22000FFF740FF4342584140B205B066
:10460000F0BD0B0ADBB2002D04D163700023A17052
:10461000E370D9E7802252421343F6E70023637028
:10462000A370F5E7FF23FAE70A0C62700A0AA2708A
:10463000002222711A0AE1706271A3710821C4E795
:104640000B0ADBB2002D09D16370130EE370130C5B
:104650002371130AA1706371A271EFE780204042B9
:104660000343F1E70B0C63700B0AA370130E237165
:10467000130C6371130AE170A371E2710921A4E7BD
:10468000C1B2B5E70020BAE7F403002042DC000025
:10469000F0B585B006000391302830D8194B1F784B
:1046A00030220023B2425B410A24FFB20293029BF4
:1046B000039A0093310004233800FFF76DFF0500D3
:1046C000012805D13800FFF7EFFE0500012813D0BF
:1046D0000120FEF7F0FD0021CF2000910B000A0021
:1046E000FFF75AFF013CCF20FFF7DEFEE4B20120C6
:1046F000FEF7E1FD002CDAD1280005B0F0BD024B39
:10470000CDE7C0463EDC00003FDC0000F0B506000F
:1047100087B00F00FF2827D81F4B1B78FF22DBB282
:1047200002930023B2425B410A250393039B0022BC
:104730000093310004230298FFF72EFF04000128A4
:1047400014D10298FFF7B0FE040001280ED1039A9D
:10475000042105A8FFF7DAFE0400012806D1059B15
:104760003B60200007B0F0BD0C4BD6E70120FEF700
:10477000A2FD0021CF2000910B000A00FFF70CFFE3
:10478000013DCF20FFF790FEEDB20120FEF793FD33
:10479000002DCBD1E5E7C04640DC000041DC000045
:1047A00013B50024CF202300220021000094FFF73E
:1047B000F3FECF20FFF778FE200016BD0020014B4E
:1047C00018707047F403002007B501A9FFF79EFF9A
:1047D00001980EBD10B5FFF799FF0023012800D006
:1047E000063B180010BD10B5FFF752FF002301284B
:1047F00000D0063B180010BD002313B51C4C01A9C6
:104800001C4801932370FFF781FF002814D0237800
:10481000002B1BD0802069464001FFF777FF00285E
:1048200022D01448FFF7D0FF702350219843014352
:104830001048FFF7D8FF07E0012301A90D482370B6
:10484000FFF764FF0028E2D1002016BD7C23502131
:10485000019A08489A4311430191FFF719FF002874
:10486000F2D001232370D5E706204042EDE7C04691
:10487000F403002024E80000F0B514000A27002605
:1048800087B003900291012C01D12600013400254C
:10489000230000952A000399C820FFF77DFE012818
:1048A00016D00120FEF707FD0021CF2000910B005C
:1048B0000A00FFF771FE013FCF20FFF7F5FDFFB2C1
:1048C0000120FEF7F8FC002FDDD10620404212E067
:1048D000C820FFF7E9FD0128E3D1002E0DD02A0002
:1048E000210005A8FFF712FE02AB1B7B029A137092
:1048F0000128D6D1002007B0F0BD32002100029877
:10490000FFF704FEF4E700000A23F0B5160089B0B3
:10491000049005910293012E00D101360027330047
:1049200000973A000499C720FFF736FE012849D1C5
:10493000C630FFF7B9FD012844D1340007AB1F8012
:10494000039080239B019C4256D8250003230B2013
:1049500004AA801810225242134303990370FFF7F0
:104960008BFD00282ED1059B2900D819FFF784FD67
:10497000002827D1244B1B78002B1DD0641BEF1976
:10498000A4B23FB2002CDCD11F4B07A81D786B1ED0
:104990009D410235A9B2FFF77BFD002812D107AB7C
:1049A0005D196B1E1B78002B0CD1023D2B78C32B9D
:1049B00008D1200009B0F0BD022107A8FFF75CFD77
:1049C0000028DBD00120FEF776FC0021CF200B0071
:1049D00000910A00FFF7E0FDCF20FFF765FD012001
:1049E000FEF769FC029B013BDBB20293002B00D077
:1049F00091E706204042DDE78025039BAD01002FB3
:104A0000A5D00223A3E7C046F4030020F0B59BB075
:104A100000911400412801D0542816D109AD00237B
:104A2000042229002000FEF73FFF00280BD16B78FD
:104A300005AA1370964B1968002904D000200121A3
:104A40001B68285698471BB0F0BD422814D109AD09
:104A50000023042229002000FEF726FF0028F2D1BF
:104A60006B7805AA13708A4B19680029EBD00020D7
:104A70001B6828560221E5E743283DD105AD0023F8
:104A80000C2229002000FEF70FFF0028DBD10920AF
:104A9000285600281FDB0823EB567E4A1B01D3183B
:104AA000DB7A04011119DBB2CB7201238B726B89A3
:104AB000083B9BB20B81784B1988013189B2198070
:104AC0001988002903D11988013189B219801B88FE
:104AD00012199BB2D380022309AA107093806B88AD
:104AE000D3806B6893606A4B19680029ABD00820AB
:104AF0001B6828560421A5E7442801D04B2821D162
:104B000009AD0023042229002000FEF7CDFE002875
:104B100000D098E700200123285605AA1070EB5614
:104B20005370002B06D16B885A49083B04019BB295
:104B300009190B81564B1968002900D183E71B68BE
:104B400005217FE74A2812D10023442209A9200029
:104B5000FEF7AAFE002800D075E7504B1A68002A1D
:104B600000D170E71B68199909A898476BE7462898
:104B700003D0482839D04D2847D1062605AD00235B
:104B8000102229002000FEF78FFE002800D05AE7EF
:104B90000C27EB89EF573F4902933B01CB18019358
:104BA00018730822AB5E6A890392698809AA518149
:104BB0006968029DD1600199C9888D421BD1002B83
:104BC00015DD00998B4212DA01259380039B34494D
:104BD0001C190D701460D0802D4B1968002900D16C
:104BE00031E71B68310038002CE70926C6E79380BF
:104BF00000230993F0E7009B102B00D823E7012343
:104C000002000100FEF750FE1DE7452803D04728AB
:104C100021D04C2821D1072609AD002308222900E4
:104C20002000FEF741FE002800D00CE700206B8832
:104C3000285605AAA9881380164B04011B19DB8886
:104C4000994200D0FFE6124B1968002900D1FAE61C
:104C50001B683100F6E60826DEE7522800D0F2E6AF
:104C600009AD0123142229002000FEF71DFE0028B3
:104C700000D0E8E60B4B6A681A601A68002A00D177
:104C8000E1E61B682A7CA96828689847DBE6C046ED
:104C9000FC1000204C100020F6030020041100201E
:104CA000E00300200011002070B5094D2C78E4B21B
:104CB000002C0CD1B02221000648FEF7F1FB06497A
:104CC0000220FEF71DFE01232B70044B1C8070BDDB
:104CD000F50300204C1000200D4A0000F6030020D0
:104CE000024B1860024B19607047C046FC10002050
:104CF00004110020F0B5170089B0022804D0012566
:104D00006D42280009B0F0BD012943D107252E4E80
:104D1000337834783078DBB201300721059303F023
:104D2000A3FDE4B2294BC9B2240131701C19A37A46
:104D3000002B2AD16B4614255D57002DE1DB102294
:104D400000212000FEF7ACFB0123A372204B1A8840
:104D5000013292B21A801A88002A03D11A880132CD
:104D600092B21A801B889BB2E380FB07C9D521232E
:104D7000E372002307AA1570502102930193009358
:104D800002200433FEF714FCBBE7013DEDB2002D19
:104D9000BED1B4E70229B2D1042303260D490E483F
:104DA0000D780C780A7824010132324024180A70F8
:104DB000A27AEDB2002A02D107356DB2BDE7013B00
:104DC000DBB2002BECD19AE7F80300204C10002056
:104DD000F6030020F9030020BC100020F0B51400F9
:104DE00089B000282DDB00292BD0174B0701DA19D9
:104DF000937ADBB2012B24D1002C22D0D47A442622
:104E0000A446654605AC1D4202D0D37A07366372CC
:104E1000207208222000FEF739FB0B4B2200DD191F
:104E2000EB883100638100230220029301930093F9
:104E30000C33FEF7BDFB002801D00920404209B029
:104E4000F0BD0620FAE7C0464C10002070B588B0CF
:104E5000002833DB002931D0AF23DB009A422DD864
:104E6000174C0601A3199D7A012D27D1DB8804ADCB
:104E7000AB8128706A805023062800DD0C3BA01906
:104E8000C67A4524F60708D50E4C038926680E48D5
:104E90009BB24C24864200D85523802004430293C1
:104EA0000192009110232A0021007E38FEF780FB3A
:104EB000002801D00E20404208B070BD0620FAE75D
:104EC0004C100020F00300203F130000F0B5070055
:104ED00087B010001A00002F29DB164C3B01E618A2
:104EE000B57AEDB2012D22D11951B0800020317B6D
:104EF00081421AD13573F07A4621284200D0073119
:104F0000002A00D1013AE418E388049204AAD3806D
:104F10000023177102200293019300930833FEF7D8
:104F200047FB002801D00E20404207B0F0BD06200C
:104F3000FAE7C0464C10002070B586B0002825DB8B
:104F4000144C050161198E7AF6B2012E1ED1CB8860
:104F500005AA538000238B72CB801070C87A492138
:104F6000304200D0053102930193009302200423C4
:104F7000FEF71EFB061E01D009267642601910229C
:104F80000021FEF78DFA300006B070BD062676428D
:104F9000F9E7C0464C100020F0B589B00592002812
:104FA0002BDB174C0701E519AE7AF6B2012E24D19E
:104FB000AA7A002A02D1002009B0F0BD6A46928A7E
:104FC0003951AA802A7B002AF5D12E73002B00D1FB
:104FD000013BE4190693E38806AAD38000231071ED
:104FE000482102930193009302200833FEF7E0FA70
:104FF0000028E1D00E204042DEE70620FBE7C04655
:105000004C1000201FB50400FEF752FAC3B2402B2B
:105010000BD8002201330292019200924A21220011
:105020000220FEF7C5FA04B010BD06204042FAE7A0
:10503000F0B599B01EAC24880591A446002800DA8A
:105040007FE0002B00D17CE03F4E05017419A77A68
:10505000F9B2012900D074E0059F022F5BD1062828
:1050600000DD6EE0E77A0F4200D16AE0012A0DD13F
:105070001868E37A002804D005991943E1720020EA
:1050800002E0059A9343E37219B0F0BD032A0AD1F6
:105090001868E27A1023002802D01343E372EEE787
:1050A0009A43E272F0E7042A0CD11B687519002BB1
:1050B00004D04023EA7A1343EB72E0E74022EB7A14
:1050C0009343F9E7022A3CD162463F2A39D8751941
:1050D000EA8806AC6280624600260225190020702C
:1050E000079208A840226570FEF7D0F9482302967F
:1050F00001960096220051212800FEF759FAC31CA0
:10510000BDD102960196009648232200D1212800A5
:10511000FEF74EFAB3E71B6806A90693E3884A71C7
:10512000CB80002308710A000293019300934F2162
:1051300008330220FEF73CFA0028A5D0092040429F
:10514000A2E70620FBE7C0464C10002073B505001F
:10515000FEF796FE294B0005000D0024984232D937
:1051600001A92748FFF742F8041E2CD1019B254EC8
:1051700025493340194322480191FFF73BF82100AC
:105180002248002D21D0FFF735F8AB212048FFF74A
:1051900031F801211F48FFF72DF821001E48FFF7C5
:1051A00029F881211D48FFF725F81D48FFF71AF857
:1051B0000128FAD18021019B49021E403143104849
:1051C0000191FFF717F8200076BDFFF713F8B9211A
:1051D0000F48FFF70FF801210E48FFF70BF82100E9
:1051E0000D48FFF707F881210C48FFF703F80C483A
:1051F000FEF7F8FF0128FAD1DCE7C0469F03000064
:1052000010140000FF8F88F800101101080201003F
:105210000C020100140201001C0201000402010042
:1052200018020100704710B5040003F01BF92000BC
:1052300010BD0000F8B504000C4B0500083308C48D
:105240009B23FF279B00C618002120002170677058
:105250002181E1612162616228301022383405F039
:1052600089F9B442F0D12800F8BDC04644DD000001
:1052700010B50400080011001A00FFF73BFD0028DC
:1052800006DB382301224343E3181A71FE325A71B8
:1052900010BD13B504AC080011001A0008CC248816
:1052A0000094FFF7C5FE16BDF7B50E001700050008
:1052B00039001A003000FFF791FD002188421BDB06
:1052C0003824022374432C19237100F00BFD019044
:1052D0002379022B0AD100F005FD019BC01A0F4B68
:1052E000984203D80020FEF77DFCF1E723790021E6
:1052F000032B03D0012323710800FEBD3823734321
:10530000A1817A88ED186A827B680A006B6130009F
:105310000B00FFF7DBFD0121EEE7C0461F4E00004A
:1053200070B5040000200D00FEF75CFC38216943D5
:1053300064182079033843425841C0B270BD70B53B
:10534000040000200D00FEF74DFC3821FD226943CA
:1053500061180B790020033B134203D10C23C85E74
:105360008B6AC01870BD382310B504005A438918E1
:10537000496902F0B1FD200010BD3823594340189F
:10538000408A7047F8B5070000200D001C00160089
:10539000FEF728FC38236B43FF183B79032B10D111
:1053A000A2B2002331002800FFF750FD002809DADF
:1053B0000E3006D1044B1878002802D1FEF712FCFB
:1053C000EEE700242000F8BDE0030020F8B50E0051
:1053D000382405000020FEF705FCFD2374432C193A
:1053E00020790338184009D10C22A35E002B05DD7B
:1053F000A081012302000100FEF756FA002338279E
:105400002371FF3363713B007343EB18186A002864
:1054100001D005F077F8774338000021EB192C30E4
:105420001962596299622818A181102205F0A2F828
:105430003000FFF781FDF8BDF7B538244C4304195F
:10544000256A06000F00002D06D1B820C00005F027
:105450004FF8A562206260623824B8217C43341979
:105460000C23E25EC90015008A4200DD0D00002019
:10547000ABB20193D30F9142434138225743F619FF
:10548000DBB2AAB2316AA068FEF70EFA0300002070
:1054900083420AD1336AB5627362A368019A5D19C7
:1054A000A389A5609B1AA3810130FEBD70B50E00D3
:1054B000382405000020FEF795FBFD2274432C19CB
:1054C0002379033B134202D00120404270BD3100DA
:1054D0002800FFF734FF0028F6D0A36A002B05D080
:1054E000382070432818436A1878EFE70C22A35E2F
:1054F000002BF5D031002800FFF79EFF0028EFD1E8
:10550000E2E7F0B587B0019000200C0004921D0086
:10551000FEF768FB38236343019AD318FD220393F7
:105520001B79033B134204D000230293029807B077
:10553000F0BD21000198FFF702FF0028F4DD85424D
:1055400000DD05000023029338336343019AD3182A
:105550000593059B9B6A002D28D0002B1BD0059B33
:105560009E6AAE4200DD2E0038276743019B320061
:10557000DF19796A049804F0E1FF7B6AAD1B9B197F
:105580007B62BB6A9B1BBB62049B9B190493029BBF
:105590009B190293DDE7039B0C229B5E002BDED060
:1055A00021000198FFF748FF0028D8D13823634332
:1055B000019AD518AB6A002BB8D1039B0C21595E18
:1055C0000029B3D10B000A002000062C05DCFFF7F0
:1055D0007DFC0020FEF706FBA8E7FFF7DDFCF8E7FF
:1055E00070B50400501E082811D802F0C3FF05133F
:1055F000101E394310104300382251436418002B09
:1056000006D01B785BB2002B02D10533237170BD2D
:105610000123FBE7382251436418002BF8D01B7894
:105620005BB2002BF4D10733F0E7002BEFD0002062
:1056300018560028EBDB3822082550432018057146
:105640000020185650432018417100215956043348
:105650004A43A418103407CB07C41B682360D6E75D
:10566000382251436418002BD2D05B787F2BCFD8DF
:105670000323CBE704201A5E002A03DC2000FFF797
:10568000A5FEC4E73822FD254A43A2181079033845
:10569000284210D1186890600425585F908106292F
:1056A00005DD1032083361CB61C21B681360200036
:1056B000FFF7C2FEABE70022012311001000FEF746
:1056C000F3F8A4E710B513000A0001000148FFF742
:1056D00087FF10BDFC03002010B5054C2000FFF72C
:1056E000A9FD044A0449200002F03CFF10BDC04659
:1056F000FC030020000000202552000070B50600C9
:105700000C008D18AC4207D0336821789B683000BC
:10571000984720700134F5E770BD7047704710B5A9
:105720000400406800F0DCFE0023237610BD10B5B5
:10573000406800F0FAFE10BDF8B5050040680C00A6
:1057400000F0EEFE2B68E7B2260A9B68012810D114
:1057500039002800FF2798472B68BC4304439B6807
:10576000310028009847030220003840184380B2D7
:10577000F8BD310028009847FF262B68000234400E
:1057800004439B68390028009847B4432043EEE760
:1057900010B5040002F066FE200010BD10B54B1CD1
:1057A0000BD0102909D0EFF3108472B6102905DD53
:1057B00002234376002C00D162B610BD0123427E45
:1057C0001A43427618224A430449891816228A56F7
:1057D0009340C2691343C361ECE7C04694DD000007
:1057E0004B1C17D0102915D0437E9B0712D4EFF322
:1057F000108272B618234B430749C9180123897DCB
:1058000049B28B40C1699943C16100D14176002AF8
:1058100000D162B67047C04694DD0000437E002B85
:1058200005D09A0704D5837E002B00D062B670475E
:10583000DB07FCD5C369024A9BB2D360F7E7C046D9
:1058400000180040037E002B04D143768376C361A9
:1058500001330376704700007FB5036902AE040090
:105860000D00029172608B4203D1828AB3889A4202
:1058700026D0200006223100103004F05FFE606860
:1058800000F045FE7379E17A013B581E8341227B8B
:1058900000936068002300F0DFFE33790021013BB4
:1058A000DBB2022B01D8074AD15C074B2A009D428C
:1058B00000D91A00606800F0FBFD606800F01DFE72
:1058C0007FBDC04654DD0000001BB70070B5182630
:1058D0000400FFF7B7FF33000821207A0D4D434342
:1058E000EB18595600F0A6FC33000821A07A434378
:1058F000EB18595600F09EFC0821607A4643AD191A
:10590000695600F097FC044B200006CBFFF7A4FF7C
:1059100070BDC04694DD0000A806002007B5437E98
:1059200000910192002B07D09A070AD5EFF310835C
:105930005A425341837672B60099019AFFF78CFF61
:1059400007BDDB07F8D5C369014A9BB29360F3E753
:1059500000180040F7B500240125194B194A5D7164
:105960001A601C71184B1948083301930360184BD7
:10597000184F4360184B194E038109233A00310038
:105980004575046104758372063B0476C472037323
:1059900002F0E8FD1248134B019A4360124B457523
:1059A00003811B233100026004613A000475837295
:1059B000183B0476C472037302F0D4FDF7BDC046F1
:1059C000A806002000093D0058DD00006806002000
:1059D000FC080020000000200A0800001D570000FD
:1059E00088060020140900201D1A000010B5024886
:1059F00002F073F910BDC046B006002013B512497D
:105A0000124800F0C5FC1249124800F0C1FC1249CE
:105A1000124800F0BDFC1249124800F0B9FC1249CE
:105A2000124800F0B5FC124C1249200000F0B0FC06
:105A300001230193023300930D220B3321000E4802
:105A400002F0C4F813BDC04600080042F40800206C
:105A5000000C0042FC080020001000420409002055
:105A6000001400420C090020001800421409002014
:105A70001C090020001C0042B0060020F7B501926E
:105A80001822162442433F4B07009B181C570091D5
:105A9000631C6ED0102C6CD03B4B3C4E1D68002D0F
:105AA00027D1290044223A4804F064FD2900442209
:105AB000384804F05FFD1022374B38491D60CA6733
:105AC000C021C120364B49005A5080001958FF357B
:105AD000A94319501A60334B334A5A800223327853
:105AE000134333707378DB09012BFBD00122264B63
:105AF0001A600125A540736900212B4373613800AA
:105B000000F098FB009B002B31D00027224B20494E
:105B10009C461B68BA00BB421DD16046013303603E
:105B20008D501C4B00999950072C19DD0123083C1E
:105B3000A4000721A140154A9B009B189A698A433B
:105B40009A61019A042A12D81000996902F012FD94
:105B50000B12141618008858A842E1D00137D9E773
:105B6000A4000023E5E70522A2400A439A61ADB2F2
:105B7000F560F7BD0422F7E70322F5E70222F3E719
:105B80000122F1E794DD0000AC090020001800407C
:105B90006809002024090020B009002004E100E089
:105BA00000E100E0000C00400540000018234343E2
:105BB000164870B5C0181623C3565A1C0FD0102BA8
:105BC0000DD001209840124B82B29A605A69114D53
:105BD00082435A61002229680F4C914200D170BD66
:105BE00093001E59864205D10C480139914203D8D1
:105BF0002960F4E70132F0E7E61876680132E650F2
:105C0000C61876681E500433F0E7C04694DD0000E5
:105C100000180040B0090020680900202409002075
:105C2000F8B50024094B1B68A34200D8F8BD084E04
:105C3000084FA5003369EA591A4204D0064BEB58C5
:105C40009847EB5933610134ECE7C046B0090020B6
:105C5000001800406809002024090020FEE7000029
:105C6000034B10B51B68002B00D0984710BDC046F1
:105C7000B409002070B50F490F4CA14204D100F0C7
:105C80008FF802F0CBFBFEE70C4D00238D42F6D0DF
:105C9000CA18E818A24205D3094B8242EFD009493D
:105CA000002204E0006804331060F1E704C38B4273
:105CB000FCD3E4E700000020A00200205CE6000026
:105CC000A00200200C11002010B500F066F800289A
:105CD00001D100F057F810BD014B18607047C04665
:105CE000B4090020014B18687047C046B80900206D
:105CF000F7B51348012284461249134C8E68636835
:105D000005689B0E1340019288686268019F920E9D
:105D10003A4067463F6893420ED1BD420CD186425D
:105D20000AD35B19FA254868AD00861B07486B4308
:105D30007043000DC018FEBD3D0013000600E3E7F0
:105D4000B809002010E000E000ED00E0555500002B
:105D500070B5041E10D0FFF7CBFF050000F01CF853
:105D6000FFF7C6FF054B401B9842F7D9FA23013CC9
:105D70009B00ED18002CF3D170BDC046E703000076
:105D80007047000010B5034A13680133136000F038
:105D9000C3FA10BDB809002070470020704700000A
:105DA0001E2270B546484749436893431C3A134343
:105DB000436008238C6923438B61434C434B9C8293
:105DC0009C8A14439C82DC681442FCD00124404A23
:105DD00014701578254203D055786DB2002DF8DB8C
:105DE00001249460547864B2002CFBDB394C54607D
:105DF000547864B2002CFBDB8224E4015480547894
:105E000064B2002CFBDB02249C840E34DD68254246
:105E1000FCD0314CDC621024DD682542FCD09D8C26
:105E20002E4C2C439C841024DD682542FCD0022497
:105E30009D8C80262C439C844024DD683542FCD018
:105E4000DD682542F9D01024DD682542FCD000240D
:105E50009460547864B2002CFBDB214C546054787D
:105E600064B2002CFBDB1C6A1E4D2C4080251C629A
:105E70001C6AAC431C62032393601B4B5360537832
:105E80005BB2002BFBDB0023FF240B72174A4B7223
:105E90008B72CB72164B1A60164B174A1B6811682F
:105EA0009A065B01C90E2340520F12020B431343A3
:105EB000124A1385802342681343436070BDC04675
:105EC00000400041000400400C06000000080040B3
:105ED000000C004001050100B905FF7D040A000027
:105EE00000070300FFFCFFFF03060100006CDC025B
:105EF00014000020246080002060800000400042E8
:105F0000FA21314B10B51868890002F03DFB2F4B88
:105F10000138984256D82E492E4A4860C020136A4C
:105F200000061B021B0A03431362002407238C6034
:105F30000B608021136A09061B021B0A0B431362C4
:105F4000FC22254B196A0A431A62FC22196A920143
:105F50000A431A62A022196AD2020A431A62E0B204
:105F60000021013400F0EEF8162CF8D11B4B1C0078
:105F70005A7852B2002AFBDB194A5A80194B1A0090
:105F8000597EC9090129FBD0E421C90099803F212C
:105F9000D970537EDB09012BFBD0C02300205B01AD
:105FA0001361907000F02EF863785BB2002BFBDB7E
:105FB0000D4B0E4A6380D379DB09012BFBD04123C3
:105FC000537010BDFEE7C04614000020FFFFFF0025
:105FD00010E000E000ED00E000040040000C004094
:105FE0001E400000004000422140000000480042E6
:105FF000914202D002D98A1AD0407047521A90407A
:10600000FBE70000164A00B51300517EC9090129BB
:10601000FBD00138042816D81969124A0A400F210A
:106020001A615A788A4302F0A5FA0308060B0300A6
:10603000110001220A435A7000BD11000322F9E742
:1060400011000222F6E7F02311691B050B430F2113
:10605000136153788B43190002230B435370EBE712
:1060600000400042FFFFFFF010B504000E2801D8E9
:106070000F34E4B20121200000F0DCF818231021D5
:1060800063432B4CE4186156002901D014290DD12B
:10609000284B1800DA79D209012AFBD002241A7899
:1060A000A2431A70C379DB09012BFBD022480300FD
:1060B000427ED209012AFBD01F2402692140A2435B
:1060C0000A4302615A7ED209012AFBD002221978C2
:1060D0000A431A705A7ED209012AFBD00222197B88
:1060E0000A431A731A7ED207FCD501221A765A7E09
:1060F000D209012AFBD00222197B0A431A731A7EA5
:10610000D207FCD5588B80B25A7ED209012AFBD027
:1061100002211A788A431A705A7ED209012AFBD0CA
:10612000064B1A68064B1968FFF762FF10BDC046A0
:1061300094DD000000480042004000421C000020A6
:1061400018000020182330B51D0004004543082026
:10615000204A55192856013014D0032912D80800B6
:106160006343D156D31802F005FA02280E1B586873
:10617000CB010221184A9B181A18403211700122D3
:1061800082405A6030BD5868CB010621124A9B18E4
:106190001A1840321170012282405A609A61F1E768
:1061A0005868CB0106210C4A9B181A18403211700E
:1061B000012282405A605A61E4E75868CB0102210B
:1061C000054A9B181A1840321170012282409A60C9
:1061D000D8E7C04694DD0000004400411823F0B524
:1061E00008245843114A13181C5701341BD00126A8
:1061F00035005F688356BD400D4ADB019A189068F0
:1062000005420BD10C00601E8441D2194032107837
:1062100034400336A400B04320431070044A9B1856
:10622000002901D15D61F0BD9D61FCE794DD0000B6
:106230000044004118224243F8B52C4E0300B21826
:10624000127A52B2140001320ED0481C00240C28DD
:106250000AD802F08FF90720202020202020200BD0
:106260000B0B0B00012464422000F8BD092905D165
:106270000021D8B2FFF766FF0024F5E70A2902D112
:10628000D8B20839F6E700240B29EDD1D8B20A3983
:10629000FFF758FFE8E718204343F2185568F35614
:1062A0002C00134ADB016E0817389B18C9B2044052
:1062B0009E19002C0DD00F2430363278090122406F
:1062C0001143C9B25B19317040331A78104318700A
:1062D000D2E732000F27303216785B19BE433143C4
:1062E000117040331A7810431870BDE794DD000038
:1062F0000044004110B50400FFF742FD014B1C6053
:1063000010BDC046200000200122024B52421A60FC
:106310007047C04620000020164A10B51368591C6B
:1063200026D0013B1360002B22D172B6124B134AC8
:106330000433934213D9124A01211000147D0C42F8
:10634000FCD02021148BFF319B085B00214311837B
:10635000D3610C4B13800123027D1A42FCD0BFF3A2
:106360004F8F094B094ADA60BFF34F8FC046FDE7F4
:1063700010BDC046200000200020000003020000E5
:106380000040004102A5FFFF00ED00E00400FA0517
:1063900000230371016070479446F0B59E1E721E83
:1063A00096416246056892072F6836063A433243A3
:1063B0002A60072505AC24780068A4012940214300
:1063C00042680024022B00D05C031143214341604A
:1063D000F0BD30B5C0250368AD031C6812052A4026
:1063E0002243C0240904A402214011431960036818
:1063F0005A6814435C6030BD0123026811680B4386
:10640000136003681A68D207FCD4DA69D207F9D49A
:1064100070470223026811680B4313600268D36956
:106420009B07FCD470470268137E9B0702D4037954
:10643000002BF9D1002303717047002203685A83AF
:1064400070470368187E4007C00F70470368187EC6
:10645000C0097047802302685B42117E0B431376AC
:1064600070470368588B8007C00F7047022302688B
:10647000518B0B43538370470368187EC007C00FCE
:1064800070470368188DC0B2704703681A7ED20740
:10649000FCD589B2198501230371180070470122C8
:1064A00003689A757047012203681A7570470000E7
:1064B00070B5012604684B08334031402568090750
:1064C0005B070B432B43236004685100034802F031
:1064D0005BF80138C0B2207370BDC046006CDC02AE
:1064E0000123026811680B43136003681A68D2071E
:1064F000FCD4DA69D207F9D4704702230268116824
:106500000B4313600268D3699B07FCD47047036890
:10651000DA699207FCD402211A688A431A6070472C
:10652000036818684000C00F70470268936A5B0AEE
:106530005B021943916203681A7E5207FCD5986A80
:10654000C0B270470368214A30B593422FD0204A29
:1065500093422FD01F4A93422FD01F4A93422FD0ED
:106560001E4A93422FD01E4A93421FD10E23192256
:106570000121032599401B48C024016099082B4044
:10658000AB40FC359D4089000918A4000859A84378
:10659000C0259D402B0003430B518023DB011A4390
:1065A000114B5A805A7852B2002AFBDB30BD0923C6
:1065B0001422DDE70A231522DAE70B231622D7E798
:1065C0000C231722D4E70D231822D1E7000800423C
:1065D000000C00420010004200140042001800426B
:1065E000001C004200E100E0000C0040F8B504008F
:1065F0000F0016001D00FFF7A5FF2000FFF7FCFEAF
:106600001C21BB000B4071072268090C0B4313606F
:10661000842322689375012F1AD11021012E00D0F6
:1066200008390C4B69431868C00001F0ADFF072220
:10663000216802408B895203DB04DB0C13438B81FE
:10664000226803049089DB0C400B400318439081BF
:10665000F8BDC04614000020F7B50600019308AB52
:106660001F780D001400FFF73BFF3000FFF76AFFB3
:10667000C022240592031440BA070C2717433C4359
:10668000C0270722BF022D0433683D4025431D600B
:10669000019B316813401A0080239B0213434B6017
:1066A000F7BD0020704770B50F26CB1D01390200E1
:1066B0003240D5B22C0000093034092A00DD0734FD
:1066C0001C70013B8B42F2D170BD000010B50C0074
:1066D0000B4B1868FFF7E7FF21000A4B08311868D9
:1066E000FFF7E1FF2100084B10311868FFF7DBFFCF
:1066F0002100064B18311868FFF7D5FF202010BD88
:106700000CA0800040A0800044A0800048A0800031
:1067100008B4024B9C46103808BC6047CD660000A8
:10672000704770473F20704713B56B460268D971B8
:106730000733546819000122A04716BD70B50A2618
:106740000B7892B06E44023305000B703C2200219E
:10675000300003F00FFF394801AC0690384824217F
:106760000790062020776846364AA1742281364A6F
:10677000364BA281FD3AFF3A8018C177684623392B
:106780000630C17768460730C17702A8C177072075
:10679000F277032608316944C87703A9CE77102120
:1067A0002B366E443170092621851F3169440E70E5
:1067B0000CA9053E0E7033212380022369440B701F
:1067C00006360DA90E7022493536A1863B216E444E
:1067D000307010A86274E27702703D3269446A44F6
:1067E0000B70137040210022E37023716371A37357
:1067F00041336B44218719705A702B7DC039A370C7
:10680000A37263770133DBB2A3776A7D0B200D009F
:1068100068441543C5773120684403703A23501CFF
:106820006B441870412302320A436B441A702100F2
:106830004222084800F0FEFC12B070BD1001042492
:10684000020605240904000001020000080B0000F4
:1068500007050000180A002008B4024B9C461038B7
:1068600008BC60473D67000070B5027D0B790C00E5
:1068700000259A420BD10B784E78A12B09D1212EFD
:1068800005D107221B491C4800F0D4FC0135280023
:1068900070BD212BFBD1202E22D10722154916488D
:1068A00000F00AFC9622134BD200196891421DD1C8
:1068B000DB79DB071AD4FA20FFF71CFD00210E4814
:1068C00000F0C0FD0125232EE1D1E378A2781B0260
:1068D00013430A4A00210848136000F0B3FDD6E7CD
:1068E000222EEFD18A78034BDA71DBE7FFF70CFD3C
:1068F000E4E7C04628000020180A002024000020F9
:1069000008B4024B9C46103808BC60476968000018
:1069100010B508220021024803F02CFE10BDC0462D
:106920002800002010B5417D006A013100F0FCFA1A
:10693000034B1B6801335A1E9341181810BDC04603
:106940003000002010B5417D006A023100F002FBEA
:1069500010BD10B5417D006A023100F0C9FA10BDCA
:1069600070B50D00417D0400130002312A00006A59
:1069700000F0B6FB002801D10123636070BD000068
:1069800010B5054C23685A1C04D103685B6998470D
:1069900003002060180010BD30000020074A0300EB
:1069A000106810B5411C03D001235B42136010BD79
:1069B000597D186A013100F043FBF8E730000020F0
:1069C00010B5FFF78FF9F423FF330024984207D95D
:1069D000044B0A20DC79631E9C41E4B2FFF7B8F94E
:1069E000200010BD280000200020704770470000E4
:1069F000FA239B0010B583600F4B0022C382030073
:106A0000283383610D4B04004260C261180050338B
:106A100023610830631D21622060DA778323A3623B
:106A2000813BE3628033236301F012FB21001031CC
:106A300001F0DFFA200010BD03020000F4E00000C6
:106A4000022110B5094B1A68437D5B01D318FF334F
:106A50009C7A21439972437D0133DBB25B01D318E9
:106A60000122FF33997A0A439A7210BDD00E00209A
:106A700010B502490248FFF7BBFF10BD180A0020FD
:106A8000BC090020704710B5040001F0EBFC2000A9
:106A900010BD0000F0B5822919D1C3B2294D5A01A9
:106AA000AA189169284C80010C40C0218905214316
:106AB00091612649083340187021506128685B01B4
:106AC0001A5C8A43110030220A431A54F0BD00298F
:106AD000FCD1C026C1B21B4C4B01E3189A681A4D79
:106AE000B6052A4032439A60194A800182185A60DA
:106AF0000A000727246808325201115DB9430F00CC
:106B00000121394311559F6910493D4040182E43DA
:106B10009E6158617020115D81430800102101437E
:106B2000115599680B48A218084080214903014378
:106B300099609968890B89039960402311790B4307
:106B40001371C3E7D00E0020FFFFFF8F440A00201F
:106B5000040C0020FF3F00F0EFF3108303600123DB
:106B6000436072B670470368002B02D162B6BFF370
:106B70006F8F704773B5836D0400002B1BD1060027
:106B8000A83635786846FFF7E7FF019BEDB2013B79
:106B900002D33578EDB2FAE768460193FFF7E3FFD9
:106BA000002D01D1002076BD2300A4331868A03445
:106BB0002368C01AF7E76846FFF7CEFF22000025DA
:106BC000019BF432013B02D31578EDB2FAE7684637
:106BD0000193FFF7C8FF002DE4D02300F0331868BD
:106BE000EC34E5E710B5436D4468DBB25A01A218F6
:106BF00091680948083308408021490301439160A6
:106C000091685B01890B890391602268D318402247
:106C100019790A431A7110BDFF3F00F0F7B5436DB3
:106C20004268DBB2190004000831106849014118BC
:106C3000C979C90711D55B01D21893689B049B0CD5
:106C40000CD12000FFF7CEFF63681A68636DDBB2DA
:106C500008335B01D3187F22DA71F7BDE16D00299B
:106C600023D12100A4310B6023000125AC33E5655D
:106C700068465360FFF770FF260020002100019B4B
:106C8000A836013BF430F5315A1C33D03570027808
:106C90005F1ED2B20A700A78002A04D12000019344
:106CA000FFF7A0FFE8E73B00EEE72100F0310B60C3
:106CB0000023E3652300603353606846FFF74CFF11
:106CC0000125260020002100019BF436013BA8305D
:106CD000F5315A1C0ED0357002785F1ED2B20A70A0
:106CE0000A78002A04D120000193FFF77BFFE8E730
:106CF0003B00EEE768460193FFF735FFA4E737B5A1
:106D00006B46DC1D00230D00237001F0A1F921006A
:106D100001F02CF92B681818286020783EBD00007F
:106D20000078002810D00121084B1B681A898A437B
:106D30001A810822198B0A431A830422198B0A43E9
:106D40001A830022024B1A607047C046D00E002002
:106D5000C80E002010B50F4A93699B0B9B039361EB
:106D600013680222FF331A729879823A02439A71A9
:106D70001A7A9207FCD57F24074A2140937A0800AB
:106D8000A3431900802301439172917A5B420B4324
:106D9000937210BDD00E00200050004110B50C00C1
:106DA00001F056F9210001F014F9002804D1034A3A
:106DB00093699B0B9B03936110BDC046D00E0020CE
:106DC000F8B50D00832A19D1CBB23B4C5A01A21859
:106DD00091693A48AD010840C0218905014391619C
:106DE000374920686D187021083355615B011A5CC2
:106DF0008A43110040220A431A54F8BD022A55D191
:106E0000304A8B009858002802D003685B69984785
:106E1000F82001F023FB0400274E2B4B4660036053
:106E200040220021083003F0A5FB22000023A032FD
:106E3000A3646565E3642365A365E3655360D36478
:106E40001372136013654C3213725372FF222B00BE
:106E50001340590171188868184F08330740C02043
:106E6000800538438860306807265B01195CAD00F7
:106E7000B1430E000321314319542300616D606852
:106E800011404901411860334B60616D63680A40ED
:106E90001B6852019B180122FF33997A20000A4394
:106EA0009A72FFF79FFE074B5C51A6E7110028007E
:106EB000FFF7F0FDA1E7C046D00E0020FFFFFF8FD7
:106EC000440A00201C0A00205CE1000070B50500A7
:106ED0000124064BA200D258002A06D02100280027
:106EE0000134FFF76DFF0A2CF3D170BDF0090020CB
:106EF0000B4BCAB20B488901C9185301C318596119
:106F000099690832890B89039961036852019A18BB
:106F10000223D3715179823B0B4353717047C046B2
:106F2000440A0020D00E0020084B8A00D05810B52B
:106F3000002803D003689B68984710BDC9B2044B72
:106F40004901591888688004800CF6E71C0A002063
:106F5000D00E002010B50C00FFF7E6FF00280CD083
:106F6000064BE4B21B68083464011C198023627963
:106F70005B42134363710223E37110BDD00E002006
:106F8000F0B51C002A4B85B01B6807000D0002926B
:106F9000002B4AD0274B8A00D058002808D003681D
:106FA00022005B68029998470400200005B0F0BDFC
:106FB0003800FFF7B9FF844204D929003800FFF7F1
:106FC000B3FF04000121EBB21B4E03935B0101935D
:106FD000F21893689B0B9B039360019A33680298A5
:106FE0009B18FF335A7A0A435A72144BA901C918E5
:106FF000220003F0A3FA002CD7D029003800FFF7B5
:1070000093FF0028D1D14021039B326808335B01F4
:10701000D3181879014319710121D971019BD31833
:10702000FF339A7A0A439A72BFE701246442BCE7AD
:10703000C80E00201C0A0020D00E0020040C0020E6
:1070400013B56B46DC1D22000123FFF799FF0128D1
:1070500001D1207816BD01204042FBE770B5CBB2CC
:10706000124A13485C01890189180219516091681C
:10707000104D08330D40802149032943402591607C
:107080009168890B8903916001685A018A18167901
:107090003543157195796D06FCD55B01C918CB791F
:1070A000DB07FCD500198068C0B270BD040C00205D
:1070B000D00E0020FF3F00F070B50D00002114003D
:1070C000FFF7CCFFA04200D9200000230349A342D0
:1070D00003D0CA5CEA540133F9E770BD040C002008
:1070E000F0B51E003A4B85B01B680F000192002BD3
:1070F00035D08023DB019E4231D80025354B8A01F3
:10710000D3180293002E2CD0334B1B680393FF231C
:107110003B401C0000930834039B64011C19A379B5
:10712000DB0921D02D4B2E49186801F02DFA2D4B8B
:107130001721584301F028FA2B4BE279920713D418
:10714000DA5D002A01D10138F7D20122DA55009B1D
:107150005A01214B9B189A69920B92039A6101255F
:107160006D42280005B0F0BD00221F4B3400DA55F7
:107170003F2E09D9009B40245A01174B9B188022AF
:10718000996912060A439A6122000199029803F054
:10719000D5F9009BA1045A010F4B890C9B18029A48
:1071A0002D195A619A69361B920B92030A439A6110
:1071B000009B039A08335B01D3180222DA715979D4
:1071C000823A0A435A71019B1B1901939AE7C04600
:1071D000C80E0020440A0020D00E00201400002019
:1071E00040420F0070110100390A002070B50D00F7
:1071F0001C000D4BAE01F61811003000220003F008
:107200009DF9EDB209496D014D196E61AB69084AEE
:1072100020001340AB61AB69A2049B0B920C9B0353
:107220001343AB6170BDC046440A0020D00E00205D
:10723000FF3F00F0F7B5104B01901B780F001500D1
:10724000002B0CD10D4B16001C78002C09D00C4ED5
:107250000C4834882018641903F070F93480280031
:10726000FEBD002EFBD03A19330000210198FFF734
:10727000BDFF2418361AF4E7C40D0020C50E002007
:10728000C60E0020C50D0020F8B50F001600002422
:10729000012A26D9100003F02BF90500380004F06C
:1072A0004BF9032302220130400028706B70964294
:1072B0000DD9397800290AD0531CDBB20137A95403
:1072C0009E4203D00232EC54D2B2F0E732002900E1
:1072D0000548FFF7AFFF441EA041C4B2280003F0E9
:1072E00011F92000F8BDC046180A0020F0B50024AE
:1072F000012685B0184B0F0069461E7005000094EA
:10730000FFF7FDFC154B01A90B806A3BFF3BCB71DE
:107310005A330B72009B8C7109334B800E4B4E71AC
:1073200008711C703A00092F0FD00D4F09223E70D2
:107330000C4E280000943480FFF77CFF694628003B
:10734000FFF7DDFC328808493C702800FFF772FF28
:10735000012005B0F0BDC046C40D002009020000A8
:10736000C50E0020C60E0020C50D002070B5CE78D9
:1073700092B005000C00022E0BD18B79C9792C48F4
:1073800009021943FFF7B2FF411E8841C0B212B093
:1073900070BD00F05DFE210000F0FCFD002803D070
:1073A000C117081AC00FF2E7012E0ED1E279A379B6
:1073B00012021A431F49112A13D8D2B2002A10D040
:1073C0002800FFF737FF0120E1E7032EDFD1A37884
:1073D000002B08D1E279A37912021A431649032A35
:1073E000EBD90A78ECE7022B08D1E279A3791202F3
:1073F00012491A432800FFF747FFC8E7012B05D1C0
:10740000E279A37912021A430D49F3E7032BBED1A7
:107410004122010001A803F0ADF800F019FE01A916
:1074200000F0C8FDE279A37912021A4301A9E1E74D
:10743000180A002098E1000088E1000078E10000CF
:107440008CE10000CBB204495B01C9188B699B0B2E
:107450009B038B617047C046D00E002037B50500F6
:1074600048780C000B2810D801F084F8061B0F2B6D
:107470000F404561494C5A5D097801AA002906D19F
:10748000022311802800FFF7B1FE01203EBD00233A
:107490001380284B1B78012B00D11370022300218D
:1074A000F0E78A780023012A03D101AA1380224B36
:1074B000F0E7204A1370214A93699B0B9B03936169
:1074C000E3E78C78012C06D100211B4B01AA1C702C
:1074D00011702300D6E70120002CD7D1154B174A95
:1074E000187093699B0B9B039361CFE78978280001
:1074F000FFF730FCC9E72800FFF738FFC6E7012394
:107500000F4ACCE70B780020DB06BFD12800FFF73D
:10751000DDFCA2780A4B0B481A60FFF791FACAE724
:107520000123094ABBE78A78074B1A60C3E70020AA
:10753000ACE7C046380A0020400A0020D00E0020E8
:10754000C80E0020BC090020CC0E00203A4BF7B535
:107550001E780500002E5FD1384C23689A8B1207E5
:107560000DD5082231009A833000FFF793FA1022DC
:107570002368FF33997A0A439A72314B1E6023685D
:107580009A8B520701D504229A83FF331A7A920606
:1075900003D52022597A0A435A721A7AD20623D581
:1075A00069460800274AC0CAC0C0A268920B92036D
:1075B000A2604022587902435A7160230A78280059
:1075C0001A422AD1FFF74AFF2368FF33002827D049
:1075D0008022997952420A439A711A7A520603D547
:1075E0004022597A0A435A727F2601252368FF33C5
:1075F0001E722F00236808377F01DB19DB79002B0F
:1076000007D0114BAA00D05800280DD003681B6882
:1076100098470135082DECD1F7BDFFF7BFFBD3E745
:1076200020210A4A9171D8E729000948FFF7DEF9BD
:107630002368DF19FE71ECE7C50E0020D00E002094
:10764000C80E0020040C00201C0A0020FF5000413E
:10765000BC09002010B50248FFF778FF10BDC046F6
:10766000180A002080235B00038000234360073357
:107670000372704783000148C0187047F00900206A
:10768000836C402B09D03F22036CC154036C01333F
:1076900013400364836C013383647047F7B50500BE
:1076A0006846FFF759FA00264022019B013B02D3AE
:1076B0002E6D961BFAE768460193FFF754FAAB6DFF
:1076C0006846002B4FD1FFF747FA2900019BA831EC
:1076D000013B5A1C0CD00C785A1EE4B2002C05D188
:1076E00068460193FFF73FFA2000FEBD1300F0E764
:1076F000684601930024FFF736FA2A002900A032D9
:107700001368A431B4420ED0086898420BD92800FF
:10771000591CEB181160603319780830C9B2FFF7B3
:10772000AFFF0134E9E709689942DDD10023136016
:107730000133AB656846FFF70FFA2F002A000021DE
:10774000019BA837013BF532581CC9D0397010781D
:107750005E1E002805D0117028000193FFF742FA41
:10776000EBE73300F0E7FFF7F7F92900019BF4316D
:10777000013B5A1C06D00C785A1EE4B2002CAFD044
:107780001300F6E7684601930024FFF7ECF92A009E
:107790002900EC321368F031B44202D008689842F4
:1077A0001DD8096899429FD1002368461360AB65D4
:1077B000FFF7D2F92F002A000021019BF437013B8B
:1077C000F532581C00D18BE7397010785E1E002806
:1077D00011D0117028000193FFF704FAEAE728009E
:1077E000591CEB181160AC3319780830C9B2FFF797
:1077F00047FF0134CBE73300E3E710B50400FFF7A0
:107800004DFF206D10BD10B50400FFF747FF236D3D
:10781000002B03D0E36CE418207A10BD0120404215
:10782000FBE7F7B517000E000400FFF737FF6846C7
:10783000FFF792F93F2200259446019B013B5A1C19
:1078400019D0BD4215D2226D002A12D00121226D1D
:107850004942002A0AD06046E26CA218117AE26C12
:1078600001320240E264226D013A22657155013510
:10787000E7E7013BE3E768460193FFF774F9280067
:10788000FEBD0000014B024A1A607047D00E002076
:10789000005000412023F7B5474A0500D1690F2069
:1078A0000B43D361012245490B7813430B70444BC2
:1078B00019788143197006211C78214319704149B8
:1078C0000C7822430A701A7802401A7060221978E4
:1078D0000A431A703C4B3D4A5A805F78FF09FCD13D
:1078E0003B48FEF7F9F901233A4C3B4E2268300041
:1078F00011780B43137080223900520002F03AFED7
:1079000022689378DB07FCD456621F26334B1B6832
:10791000590B980C9B01314030405B0FB14200D1B4
:1079200005211F2800D10238072B00D1043B31402C
:107930008901178D01912A4930400F40019939433F
:107940001185118D0700B143080038431085118D52
:107950001803244B7F260B4003430C201385082378
:10796000D17881430B430321D3702268D3788B43B2
:1079700001390B43D370226813783340137004230A
:1079800022681678334313702268C1241389A40037
:1079900083431548138103591B021B0A035180239B
:1079A0000360137811481943012311702B700021D3
:1079B000FEF7B6FEF7BDC046000400405844004143
:1079C0003C44004159440041000C00400640000086
:1079D00055760000D00E0020D40E002024608000D8
:1079E0003FF8FFFFFF8FFFFF00E100E0BC09002030
:1079F0000120704710B50368014A1B6A984710BD03
:107A000013040000FC30006A704787239B00C018F5
:107A1000C36880204000C01A70470300FC331A6A14
:107A2000002A03D0DB69C018007D70470120404266
:107A3000FBE710B504000069FEF7DEFC220000231E
:107A4000FC329361D361136287229200A4186360B1
:107A5000A360E36010BD872310B59B00C218D368F4
:107A6000002BFCD10069FEF7DEFC10BDF0200140C8
:107A70003039484248417047F0231B0119408023A8
:107A800006209B0099420AD00133FF33013099420E
:107A900005D0802302385B00994200D00020704757
:107AA0000F2001400020012903D00239481E8141E6
:107AB000481C70478B23F0B5182685B002919B00B7
:107AC0000400C05C330008214343324D1700EB181B
:107AD0005956FEF7AFFB304B0821E05C33004343BF
:107AE000EB185956FEF7A6FB2C4BE25C0393022AD7
:107AF00009D11133E05CFF2805D008214643AE19B7
:107B00007156FEF797FB8C26B600A05DFF2819D0B2
:107B10000121FEF717FB1822A35D21495A43AB56FA
:107B2000AD18DB0158188D21890060501D490122D4
:107B30005B188E218900635069688A408F21890013
:107B400062501A600122029B11002069FEF74EFD6F
:107B500039002000FFF790FF390005002000FFF7F3
:107B60009FFF390006002000FFF780FF33000090E0
:107B7000290020690122FEF70FFC0B4B2069E25C13
:107B8000039BE15CFEF725FC2069FEF742FC05B093
:107B9000F0BDC04694DD00002D0200002F02000061
:107BA00018440041144400412E020000802210B508
:107BB00004005200002102F0DDFC23000022FC330F
:107BC0005A6020009A60DA6010BD0000F7B51D0011
:107BD00008AB1B780400009309AB1B7816000193D7
:107BE00000234360FA239B008360114B0F0008338E
:107BF00003601430FFF7DAFF20002130FF30FFF779
:107C0000D5FF8B236A469B002761E654094B127807
:107C1000E554094B2000E2546A46084B1279E254BD
:107C20008C22313BFF3B9200A3541032A354FEBD83
:107C3000ACE100002D0200002E0200002F02000027
:107C4000F7B5EFF3108300930123019372B68026FA
:107C50000200FF25019BFC327600013B5C1C0FD02B
:107C6000D4685F1EB44209D0546801555468013489
:107C70002C405460D4680134D460EEE73B00EDE75B
:107C800068460193FEF76FFFF7BD13B5EFF310835E
:107C900000930123019372B6019B5A1E0192002B9F
:107CA00015D00300FC33DA68002A0DD09A68845C92
:107CB0009A680132D2B29A60DA68013ADA606846AC
:107CC000FEF751FF200016BD01246442F7E70124AE
:107CD0006846FEF748FF6442F4E710B50400006907
:107CE000FEF7BFFB002805D02069FEF7CAFB20691C
:107CF000FEF7BCFB2069FEF7A4FB00281BD020691F
:107D0000FEF7BFFB010020001430FFF799FF8C2322
:107D10009B00E35CFF2B0ED02300FC331A6A802308
:107D20005B009B1A092B06DC8D238F229B0092009F
:107D3000E358A2581A602069FEF79EFB00280ED077
:107D400087239B00E318DB68002B14D02000213030
:107D5000FF30FFF79AFFC1B22069FEF796FB20695A
:107D6000FEF774FB002805D02069FEF773FB20693D
:107D7000FEF763FB10BD2069FEF795FBEFE70000FF
:107D8000F8B5040000690D00FEF776FB87239B0021
:107D9000E618002802D0F368002B34D00127802297
:107DA000F3685200934223D1EFF310833B4210D18A
:107DB000174B5B68DB05DB0DF1D0103B5BB2002B92
:107DC00010DAF13A1340083B9B08124A9B009B18BB
:107DD0001B682069FEF750FB0028E0D02000FFF769
:107DE0007CFFDCE79B08C0330B4A9B009B58F0E705
:107DF00020002130FF302900FFF722FF2069FEF725
:107E00004EFB0120F8BD29002069FEF73EFBF8E794
:107E100000ED00E01CED00E000E100E010B5040022
:107E20001430FFF732FF8C239B00E35CFF2B0ED056
:107E30002300FC331A6A80235B009B1A0A2B06DDA1
:107E40008E238F229B009200E358A2581A6010BD27
:107E500010B51C00431A0298511A001B584300F039
:107E60001DFC001910BDF7B5C31D019300230600CA
:107E70000D00041D009321780A22280000F0A3F9C8
:107E80002E210700280000F029F9009B3F18DB197C
:107E90000093019B01349C42EDD1F17928000A2224
:107EA00000F091F9009B1818FEBD0000024B08334A
:107EB0000360002343607047E0E1000030B503AC8D
:107EC0002578044CC57108340460017142718371D6
:107ED00030BDC046E0E10000024B41600833036062
:107EE0007047C046E0E10000F0B50124644206009E
:107EF000002527000A200B78002B20D01A00303AEA
:107F00000131092A0FD89BB2621C02D1303B1CB24E
:107F1000F1E7220042439A18303A92B214B2FF2A93
:107F2000E9D9002012E02E2BFBD1032DF9D0631CE0
:107F3000F7D06B1C75192C71DDB23C00DBE7180023
:107F4000032D03D1631C01D00120F471F0BD416009
:107F500070470000034B044A08331360002353604A
:107F60007047C046E0E10000D40F002070B50E005D
:107F700000254468002C0BD0236831005B6820008A
:107F80009847002802DB2D18E468F3E701256D42CD
:107F9000280070BD70B50D004468002C08D023681F
:107FA00029009B6820009847002802D1E468F4E784
:107FB000200070BD70B50D004468002C07D0236808
:107FC00029002000DB689847E4682D18F5E72C703D
:107FD00070BD70B50D004468002C08D023682900DE
:107FE0001B6820009847002802D1E468F4E72000CD
:107FF00070BDF8B542788B790D00017A9B180400AA
:1080000000208B4222DC6368834219D16560002620
:1080100023786A71EA792B719B182370AB79B3428C
:1080200013D9AB68B7006078DF19FFF723FB3B6813
:10803000013603606378F6B201336370EEE70B003C
:10804000D9680029FBD1DD60E1E70120F8BD00001F
:1080500070B50126054D064C2B68334203D1200034
:10806000FFF700FB2E60200070BDC046DC0F002033
:10807000E00F0020F7B506000D000C008B180193EF
:10808000019B671B9C4207D0336821781B68300036
:10809000984701340028F3D13800FEBD70B50400C4
:1080A00008000D0003F048FA2368020029005B680D
:1080B0002000984770BD10B50B1E02D0FFF7EEFFF1
:1080C0000300180010BD10B503688A685B68096872
:1080D000984710BD10B5FFF7EEFF10BD10B503684F
:1080E0001B68984710BD000010B50249FFF7D6FF86
:1080F00010BDC046ECE1000070B50500FFF7E3FFDE
:1081000004002800FFF7F0FF201870BD70B50400D0
:10811000FFF7D1FF05002000FFF7E6FF401970BD13
:10812000F0B58BB06B461500002205330600DA77F8
:108130000800012D00D80A2509AC290000F0AAFA90
:10814000CAB2130037330700DBB2092902D8130083
:108150003033DBB2013C2370002FEED12100300020
:10816000FFF7A9FF0BB0F0BDF8B506000C00151E17
:1081700004D10368C9B21B689847F8BD0A2A0CD11C
:1081800000290BDA2D21FFF7A9FF614207002A0021
:108190003000FFF7C5FF3818EFE7D2B221003000FA
:1081A000FFF7BEFFE9E710B5FFF7DEFF10BD10B522
:1081B000002A04D10368C9B21B68984710BDD2B227
:1081C000FFF7AEFFFAE710B5FFF7F1FF10BD10B5EE
:1081D00004000068002801D002F094F9200010BDCE
:1081E00010B504000068002801D002F08BF90023CC
:1081F0002360A360636010BD70B504000D000068CB
:10820000013103F04BF9031E01D0012028C470BDD9
:10821000036810B50400002B04D043688B4201D3DF
:10822000012010BD2000FFF7E7FF0028F9D0A36868
:10823000002BF5D122681370F2E770B50E00110023
:1082400004001500FFF7E4FF002804D12000FFF729
:10825000C7FF200070BD2A003100A560206802F031
:108260006DF900232268A1685354F2E7002370B52A
:1082700004000D00036043608360994207D008004A
:1082800003F05AF9290002002000FFF7D6FF200072
:1082900070BD70B5050008000C0003F04DF9210019
:1082A00002002800FFF7C9FF70BD10B500230400CD
:1082B0008AB023606360A360080001A900F04EF952
:1082C000200001A9FFF7E5FF20000AB010BD10B59E
:1082D000002304008AB023606360A360080001A942
:1082E00000F011F9200001A9FFF7D3FF20000AB028
:1082F00010BD10B50B000400884205D009680029A4
:1083000004D09A68FFF799FF200010BDFFF768FFBF
:10831000FAE7002310B50400036043608360FFF7B1
:10832000E8FF200010BD10B50400002903D0FFF7BE
:10833000B0FF200010BDFFF753FFFAE730B5D5B00E
:10834000190058AB040010001A7800232360636002
:10835000A360131C0A2A00D90A23DBB29A1C03ADBE
:1083600052B2009500F082F801002000FFF7DBFF19
:10837000200055B030BDF7B504000F0016000029ED
:1083800003D1002301930198FEBD01230193002A2C
:10839000F9D08368D5182900FFF73AFF0028F0D0FC
:1083A0002368A26839009818320002F0C7F800224A
:1083B0002368A5605A55E6E770B5050008000C0073
:1083C00003F0BAF8210002002800FFF7D4FF70BDC7
:1083D000002310B5994202D0FFF7EEFF030018000A
:1083E00010BD10B58A6809680400FFF7C4FF0028B3
:1083F00002D12000FFF7F4FE200010BD10B50400EC
:10840000002904D12000FFF7EBFE200010BDFFF78C
:10841000DFFF0028F6D0F8E77047000010B5FDF741
:108420006FFD02F02FF8FFF7F7FF0120FDF790FC3A
:10843000084C2000FFF72EFA2000FEF771FCF9F738
:10844000F1FFF9F7F5FE044B002BFAD000E000BF76
:10845000F7E7C046180A00200000000010B502F03F
:1084600047F810BD10B502F04DF810BD30B504004E
:1084700087B00D00064901A803F02CF822002B005C
:1084800001A90A9803F026F80A9807B030BDC04643
:10849000EFE10000F0B50C008BB01600002926D0EB
:1084A000931E222B2DD80A2A05D1002803DA012792
:1084B000404201AD0AE00027FBE7310000F0EAF896
:1084C000CBB2092916D830332B7001352A00002889
:1084D000F3D101ABAB42F0D02300002F02D02D210D
:1084E000631C217001A98A4206D800221A7020005C
:1084F0000BB0F0BD5733E7E7013A1178197001333B
:10850000F0E70024F3E7F0B50D008BB01700002969
:108510000ED0931E222B1FD801AC2600230000286A
:1085200009D1A64207D02A00B34210D80023137005
:1085300028000BB0F0BD390000F0ACF8CBB209292F
:1085400003D8303323700134E8E75733FAE7013BAF
:10855000197811700132E7E70025E9E710B5FFF758
:1085600099FF10BD0B0010B50100180001F07CFF51
:1085700010BD000002B4714649084900095C490079
:108580008E4402BC7047C046002243088B4274D31D
:1085900003098B425FD3030A8B4244D3030B8B4204
:1085A00028D3030C8B420DD3FF22090212BA030C0D
:1085B0008B4202D31212090265D0030B8B4219D3EE
:1085C00000E0090AC30B8B4201D3CB03C01A52410E
:1085D000830B8B4201D38B03C01A5241430B8B4256
:1085E00001D34B03C01A5241030B8B4201D30B033F
:1085F000C01A5241C30A8B4201D3CB02C01A524166
:10860000830A8B4201D38B02C01A5241430A8B4228
:1086100001D34B02C01A5241030A8B4201D30B0211
:10862000C01A5241CDD2C3098B4201D3CB01C01A2B
:10863000524183098B4201D38B01C01A5241430935
:108640008B4201D34B01C01A524103098B4201D323
:108650000B01C01A5241C3088B4201D3CB00C01A90
:10866000524183088B4201D38B00C01A5241430808
:108670008B4201D34B00C01A5241411A00D201462D
:10868000524110467047FFE701B5002000F0F0F8B6
:1086900002BDC0460029F7D076E7704703460B437A
:1086A0007FD4002243088B4274D303098B425FD3EB
:1086B000030A8B4244D3030B8B4228D3030C8B4217
:1086C0000DD3FF22090212BA030C8B4202D31212FD
:1086D000090265D0030B8B4219D300E0090AC30BD2
:1086E0008B4201D3CB03C01A5241830B8B4201D37F
:1086F0008B03C01A5241430B8B4201D34B03C01A68
:108700005241030B8B4201D30B03C01A5241C30ADF
:108710008B4201D3CB02C01A5241830A8B4201D350
:108720008B02C01A5241430A8B4201D34B02C01A3A
:108730005241030A8B4201D30B02C01A5241CDD2DF
:10874000C3098B4201D3CB01C01A524183098B422A
:1087500001D38B01C01A524143098B4201D34B0113
:10876000C01A524103098B4201D30B01C01A524176
:10877000C3088B4201D3CB00C01A524183088B42FD
:1087800001D38B00C01A524143088B4201D34B00E6
:10879000C01A5241411A00D2014652411046704758
:1087A0005DE0CA0F00D04942031000D3404253405D
:1087B00000229C4603098B422DD3030A8B4212D31D
:1087C000FC22890112BA030A8B420CD3890192114F
:1087D0008B4208D3890192118B4204D389013AD08C
:1087E000921100E08909C3098B4201D3CB01C01A61
:1087F000524183098B4201D38B01C01A5241430974
:108800008B4201D34B01C01A524103098B4201D361
:108810000B01C01A5241C3088B4201D3CB00C01ACE
:10882000524183088B4201D38B00C01A5241D9D2E6
:1088300043088B4201D34B00C01A5241411A00D267
:108840000146634652415B10104601D34042002B63
:1088500000D54942704763465B1000D3404201B5E2
:10886000002000F005F802BD0029F8D016E7704797
:108870007047C0468446101C62468C46191C6346ED
:1088800000E0C0461FB500F0F1FE002801D4002131
:10889000C8421FBD10B500F049FE4042013010BD76
:1088A00010B500F0E3FE002801DB002010BD012020
:1088B00010BDC04610B500F0D9FE002801DD002033
:1088C00010BD012010BDC04610B500F06BFE0028A1
:1088D00001DC002010BD012010BDC04610B500F025
:1088E00061FE002801DA002010BD012010BDC04645
:1088F000F0B54F464646D6460C000903C0B5490AB6
:10890000470F5E0039431F03DB0F9C4665007B0A5F
:10891000570F1F436D0DE40F760DA146C000B846FA
:10892000D200AB1B64457BD0002B5FDD002E00D056
:10893000A4E03E00164300D112E15E1E002E00D0DE
:108940009EE1871A4346B84280410125C91A404238
:10895000091A0B0200D431E149024E0A002E00D15F
:108960006EE1300001F062FD0300083B1F2B00DDCB
:1089700061E120223900D21A9E40D1409F400E432F
:108980009D4200DD51E15D1B6B1C1F2B00DD7CE176
:108990002021C91A3D0030008F408840DD40791EFB
:1089A0008F41310007222843D940002507433A4030
:1089B000002A09D00F233B40042B05D03B1DBB42AE
:1089C000BF417F42C9191F000B0200D426E26A1C76
:1089D000C64B55056D0D9A4200D106E1C44AFF0809
:1089E0000A40530752023B43120B8EE0002B00D08B
:1089F000B8E06B1C5B055B0D012B00DC30E1871AD6
:108A00004346B842B641CB1A76429E1B330200D58C
:108A10004CE13B003343A1D100220024002570E04B
:108A2000002B00DCE5E0002E00D183E0AF4EB54224
:108A300060D0802636043743B846382B00DC3EE150
:108A4000434613431F007A1E97413F1887428041D7
:108A5000404209180B0200D4B0E0A44B01359D42FE
:108A600000D1C3E0A24A7B080A4001210F401F4306
:108A70005108D30707221F433A4099E79B4EB5425E
:108A800038D0802636043743B846382B00DDDCE08A
:108A90001F2B00DC30E11E004746203EF740BC465D
:108AA000202B04D04026F31A46469E40324317003E
:108AB00063467A1E97411F43CCE0002B00D104E2AD
:108AC0004346134300D159E14B07C00818438023A4
:108AD000C9081B03194208D04546ED081D4204D1C0
:108AE0004346D008590708432900420FC9007F4D6B
:108AF0001143C0004B07CA087C49C00803438D429C
:108B000068D012036D05120B6D0D002112031800C1
:108B1000130B0A0D12051A43764B2D0513402B43F8
:108B20005B00E4075B08234319001CBC9046994690
:108B3000A246F0BD3E00164312D05E1E002E00D0AD
:108B400000E18718874280414144404209180125CD
:108B50000B0233D5022585E76446330041461000F9
:108B60001D00C7E7002D00D0DAE00C000443F3D06D
:108B70005C1C00D19FE15D4CA64200D12FE1DB439C
:108B8000382B00DD66E11F2B00DD83E1202405008A
:108B9000E41A0F00DD40D940A0404346A7405B1ACD
:108BA000441EA04198462F433843171ABA429241B7
:108BB00043465242991A64463500CAE607223A40B3
:108BC000002A00D0F6E64B07CA084849FF083B4395
:108BD0008D4296D11900114300D19EE180210903F5
:108BE0000A431203120B414D8FE7150000220023A8
:108BF0008BE7002B00D0C7E06B1C5F057F0D012FBA
:108C000000DCF1E0394DAB4200D1B9E085180A0033
:108C1000854289414244494251180722CF076D08D5
:108C20002F4349083A401D00C2E607223049ED1A99
:108C300031403A40BCE63E002838864000279FE697
:108C4000380001F0F3FB20308EE6434613431F004B
:108C50007A1E9741C71BB84280414042091A78E604
:108C60000E003B0006431343002D61D1002E00D0BF
:108C7000F4E0002B00D11BE164463900100039E715
:108C80001A4FBB427AD03300FFE630001F3DE84068
:108C9000202B03D04021CB1A9E4037437B1E9F419F
:108CA000072207433A400021002589E7171A434667
:108CB000BA42B641591A76428E1B64464EE61F2BC5
:108CC00000DDADE020264746F61AB740B94617004A
:108CD000B246DF404E463E4337005646B240561E2F
:108CE000B24117434246DA408918AEE6FF0700005A
:108CF000FFFF7FFFFFFF0F8020264746F61AB74091
:108D0000B9461700B246DF404E463E43370056464E
:108D1000B240561EB24117434246DA40891A99E7DB
:108D20007F4CA6425BD0802424045B42214327E78A
:108D3000002E0CD1002B00D1CBE06446390010008E
:108D4000774DD7E6764FBB4218D0330075E6002B3F
:108D500014D04B07C00818438023C9081B031942CD
:108D600007D0FC081C4204D17907D0080843E1462B
:108D700021004C46420FC9001143C000684DB9E6BE
:108D80001D0000220023C0E6002D5BD10D0005432D
:108D900000D1E2E65D1C00D1B0E0614DAE421FD0D3
:108DA000DB43382B71DC1F2B00DD96E020250F0004
:108DB000ED1AAF40B9460700AA46DF404D463D4395
:108DC0002F005546A840D940451EA8418844074376
:108DD000BF18974292415142414435003AE66446F9
:108DE00035004146100085E60B000343002D00D0FE
:108DF00063E6002BF5D04346134300D17AE687188B
:108E00008742804107224144404209183A400B0200
:108E100000D4D5E6434B01351940C9E5380069E671
:108E20001E004746203EF740BC46202B04D040267B
:108E3000F31A46469E403243170063467A1E974116
:108E40001F4302E6364DAE42CAD080252D045B4258
:108E50002943A6E70843411E8841A6E6002B00D11E
:108E600048E6871A4346B842B641CB1A76429E1B63
:108E700033024BD5171A4346BA429241591A52420D
:108E8000891A072264463A4092E501430F00791E91
:108E90008F419DE71C000F00203CE740202B03D0B2
:108EA0004024E31A99400843411E884138437CE638
:108EB0000022002425E6171A4346BA429241591A65
:108EC0005242891A6446350043E541461000144D6C
:108ED00010E680220024120380E61D000F00203DD2
:108EE000EF40BC46202B03D04025EB1A99400843A5
:108EF00007006346781E87411F4369E7871897423A
:108F00009B4141445B42C9183500A3E53B00334314
:108F1000CED0072231003A4052E600231A00F4E591
:108F2000FF070000FFFF7FFFF0B55746DE464E46C5
:108F30004546E0B5834607000E03480085B09246DB
:108F40001C00360B400DCD0F002800D19DE0954B45
:108F5000984239D08023F6001B041E43924A7B0FAF
:108F6000334399469446030063440093002300264C
:108F7000FF00029323031B0B98466300E40F524645
:108F80005B0D019400D1B3E086498B4200D19EE095
:108F90004246D100802212040A435146490F114330
:108FA0008B46814952468C4600996344CB1A002176
:108FB000D20000932B0063409A460F2E00D905E1A2
:108FC0007A4BB6009B599F465B463343994600D087
:108FD000B8E002230826002700900293CAE7CB4698
:108FE0003A0002990195019B9A46022927D003294C
:108FF00000D180E2012944D06D49009B8C46634436
:109000001C00002C38DD530700D013E2D2085B4669
:10901000DB0109D55946674B19408B468021C900B1
:109020008C46009B63441C00634B9C4207DC5B4600
:1090300064055F075B0217431B0B620D02E0002310
:109040000027584A00211B031C0B0B0D1B05234353
:1090500014055A4A380013401C4353466400DB078A
:1090600064081C43210005B03CBC90469946A246CA
:10907000AB46F0BD0122524201231B1B382B00DC02
:10908000ADE1002200230027DCE75B46334399462D
:109090005ED0002E00D18AE1300001F0C7F9030054
:1090A0000B3B1C2B00DD7BE11D22D31A5A4601002D
:1090B000DA4008398E4013005F46334399468F40AB
:1090C0003F4B00261B1A00930023029352E74146B0
:1090D00053460B433B499B468C46009B634400939D
:1090E0005B46002B3BD1022300221E43022161E795
:1090F000434613439B4637D04346002B00D162E1E1
:10910000404601F093F903000B3B1C2B00DD53E1BB
:1091100002004146083A914088461D21CB1A51462B
:10912000D9400B0041460B439B46534693401A00DF
:10913000009B25499C46604403008C466344009391
:10914000002137E70323B14600900C26029311E774
:109150000023009301330426002702930AE7032328
:10916000C3461E43032125E701331E43002201218C
:1091700020E700239A46802300271B03094A61E762
:10918000802349461B03194200D1E2E059461942A7
:1091900000D0DEE00B431B0317001B0BA246014A65
:1091A00050E7C046FF07000001FCFFFFF8E10000A8
:1091B000FF030000FFFFFFFEFE070000FFFF0F8020
:1091C0000DFCFFFF01F8FFFFF3030000D94500D9B4
:1091D000CBE000D1C6E03C0048460027009B013BA5
:1091E00000935B46160E1B021E431302984633047F
:1091F0001B0C9946310C0191FFF74CFA4A46424349
:109200000B04210C050019438A4207D98919013D35
:109210008E4203D88A4201D9851E8919881A01997C
:10922000FFF738FA09048C464A4621046446424353
:10923000090C030021438A4204D98919013B8E425B
:1092400000D8F1E02D041D43AB464346891A42463F
:10925000280C12041D0C5B46140C22001B041B0C72
:109260005A4303946B434443029568431B19150CFE
:10927000EB189C4203D980246402A44660441C0C71
:1092800015041B042D0C20185D19814277D373D06F
:109290000C1AA24A7D1BAF42BF419446009B7F42FD
:1092A0006344E01B1C00864200D1DBE00199FFF71C
:1092B000F1F94A4642430B04290C070019438A423C
:1092C00007D98919013F8E4203D88A4201D9871EE6
:1092D0008919881A0199FFF7DDF909044A46894678
:1092E00029044D464243090C030029438A4207D909
:1092F0008919013B8E4203D88A4201D9831E8919FC
:109300003F04891A3A00039F1A43380013041B0CC8
:10931000584381460298150C6F43434345434846E2
:10932000000C8446DB1963449F4203D9802040022D
:109330008446654448461F0C00041B04000C7D193C
:109340001818A94200D284E000D17FE001231A431B
:1093500057E680234A461B0313431B031B0BAA46F5
:109360006F4A6FE6BA4200D935E74B46DC0758082A
:109370007B081C43FF0734E70024AF4289D24744EF
:109380004745A4415B466442A4196418013BA642C8
:109390001ED2A0426DD800D1B6E0241A9B4678E7D1
:1093A00003005A46283B9A400027914688E65846D3
:1093B00001F03CF8203072E603005246283B9A4008
:1093C00093460022B4E6504601F030F820309AE689
:1093D000A642E2D1B845DCD9341A9B4659E71F2B87
:1093E00065DC504C0099A4465C46614408008C4002
:1093F00011008240D940501E82410C4314435A460A
:10940000DA401300620709D00F222240042A05D057
:109410002200141D9442894149425B181A0262D508
:109420000122002300270DE68A4200D80AE7831EA6
:10943000891907E70F231340042B00D1E6E5171D18
:109440009742924153429B44FA08E0E5002800D13C
:10945000D7E57118531EB14227D3A94215D358D06E
:109460001A0073E7002B00DC04E6012300229B4472
:10947000CDE502234744474589415B429C4649422A
:1094800089190C19E344241A03E743465F00474552
:109490009B41B8465B429E19023A8919A94200D005
:1094A00054E7404500D051E7ABE51A00F6E71F212D
:1094B0005F4649420C1BE740202B07D01A49009B0E
:1094C0008C46634418005B4683401A43501E824119
:1094D0003A4307270023174009D00F2100231140EA
:1094E0001400042995D122005F075B021B0BD208F0
:1094F00017430022A6E5802359461B030B431B0399
:1095000017001B0B064A9DE5BD42B2D89B460024BE
:10951000BFE68045B9D31A00C3E7C046FF03000089
:10952000FF0700001E0400003E040000F0B54F4697
:109530004646D6468446C0B58046194E18030F03EA
:109540004D00000B5C0082463F0B6D0DC90F91462C
:10955000640DDB0F0120B5420AD0B44203D0A5420E
:1095600001D157450CD01CBC90469946A246F0BD8F
:1095700066463E43F7D1AC42F5D154461443F2D18E
:109580000120C845EFD1994207D0002DEBD16346A9
:109590001F433800471EB841E5E70020E3E7C04617
:1095A000FF070000F0B54F464646D6464D00C0B511
:1095B0000E03C90F8A462C491F035C008046360BF8
:1095C0006D0D91463F0B640DDB0F8D421ED08C421A
:1095D00016D0002D1ED130438446002C01D13A43D1
:1095E00023D06246002A1AD09A4529D0514602203B
:1095F0000139084001381CBC90469946A246F0BD8E
:1096000039001143E5D002204042F4E73043FAD15B
:10961000AC420FD0002C0FD13A43E7D00CE001222E
:10962000013B934318000130E5E763460020002B1F
:10963000E1D0DBE73A43E6D19A45D7D1A542D5DC64
:10964000A54205DBBE42D1D808D00020BE42D2D20E
:1096500050460123013898430130CCE7C845C5D8AE
:109660000020C845F4D3C6E7FF070000F0B54F4619
:109670004646D6464D00C0B50E03C90F8A462E4950
:109680001F035C008046360B6D0D91463F0B640D49
:10969000DB0F8D4218D08C4211D0002D18D13043F1
:1096A0008446002C1ED13A431CD163460020002B77
:1096B00030D0514602200139084001382AE03900F3
:1096C0001143EAD0022025E03043FBD1AC4226D042
:1096D000002C26D13A4324D15146022001390840BA
:1096E000013817E06246002A0FD09A45E1D1A54221
:1096F00005DBBE42DDD819D00020BE420AD250465A
:10970000012301389843013004E00122013B9343D7
:10971000180001301CBC90469946A246F0BD3A4361
:10972000D0D19A45C5D1A542C3DCE0E7C845C0D831
:109730000020C845E3D3EDE7FF070000F0B557462A
:10974000DE464E464546E0B5834606000F03480018
:1097500087B092461D003F0B400DCC0F002800D172
:109760006FE0DE4B984238D08023FF001B041F437C
:10977000730F3B430193DA4B0027994600239B4626
:10978000F60081442B0369001B0B52469846490D95
:10979000ED0F002900D185E0D04B994200D173E054
:1097A0004346DA0080231B0413435246CC48520F31
:1097B00084461343524600206144D200894421006C
:1097C000694000918C46012149448A460F2F00D9F7
:1097D00090E0C449BF00CF59BF465B463B4301936D
:1097E00000D06AE102230827002681469B46C9E78C
:1097F00032005846019B61460091022800D175E075
:10980000032800D1FEE1012800D02CE1002300272D
:10981000002600253F032A0D3F0BB34812053A43AB
:1098200002401B051343009A5B00D1075B080B4302
:109830003000190007B03CBC90469946A246AB46A2
:10984000F0BD5B463B43019300D12FE1002F00D1D7
:10985000A5E1380000F0EAFD03000B3B1C2B00DD06
:1098600096E11D22D31A5A460100DA405E460839B5
:109870008F4013008E403B4301939C4B00271B1AE3
:10988000994600239B467DE7414653460B43934947
:109890008C46E144002B00D01AE10222022017433B
:1098A00000228CE7134300D10DE14346002B00D189
:1098B00081E1404600F0BAFD02000B3A1C2A00DDAF
:1098C00072E10100434608398B4098461D239A1ADD
:1098D0005346D3401A004346134352468A404946F2
:1098E000081A824989468144002068E77B4B00279B
:1098F00000268EE7140C1204120C1100370C3604EB
:10990000350C794328008C462E0060436044834622
:1099100056432100300C804658467943404402911A
:10992000844506D98846802149028C46E044414658
:1099300002913604010C360C00048B4681191E0C72
:109940001B041B0C0391190079438C4628007543B6
:109950006544A8465843050C45447743A94203D9BA
:10996000802149028C466744290C8C46390000044A
:10997000000C2D042D186144AB4405915946049107
:1099800001990F043F0C080C3900514342439046A3
:1099900002008C46090C8B4662437C4344445C4481
:1099A000A04503D98021490288464244210C8846BB
:1099B00061460904090C8C463900594343437043FE
:1099C0007E430F0CF6182404BE19644442448C46AE
:1099D000B34203D980235B0298464044029B614610
:1099E0009846049B370443449B46AB45AD416B42CC
:1099F0000D0405992D0C8C467F196744FD18A84667
:109A00005D462D19A542A44193466442A446C34431
:109A1000DC448F42BF4198459B4193459241A44508
:109A2000A4415B427F421F43360C52426442BF193D
:109A30002243BF18624638184302D20D03991343DC
:109A40006A020A43501E82416146ED0D2A434E02CE
:109A50003243D90100D4B3E001265008324002431A
:109A6000DE0732435B08224C5444002C62DD510770
:109A700009D00F201040042805D0101D90429241BB
:109A800052429B180200D90104D580241948E400F1
:109A9000034054441848844200DD27E75E075B0218
:109AA000D2081F0B630516435B0DB2E600239946EF
:109AB0000133042700269B4664E603230197814671
:109AC0000C279B465EE6012201201743002276E622
:109AD000032303201F43434671E6C046FF070000EF
:109AE00001FCFFFF38E20000FFFF0F800DFCFFFFCD
:109AF000FF030000FFFFFFFEFE070000002380279A
:109B000000933F030026434B83E6019B3200A446AB
:109B1000584670E6AC466EE6802701993F0339420D
:109B20002DD03B422BD11F433F033F0B0095160026
:109B3000384B6EE601252D1B382D00DD66E61F2D06
:109B400040DC35481C005044160082408440EE4002
:109B5000501E824134431443EB40620709D00F2268
:109B60002240042A05D02200141D94428041404224
:109B70001B181A023ED501230027002649E680273C
:109B8000019B3F031F433F033F0B0094214B40E6E3
:109B900003005A46283B9A40002601926DE658463B
:109BA00000F044FC203057E603005246283B9A4020
:109BB0001300002293E6504600F038FC20307BE68C
:109BC000CA4650E71F201E004042041BE640202DDD
:109BD00003D0124C5444A3401A43501E82413243D6
:109BE00007260027164009D00F200023104014003C
:109BF0000428B9D122005E075B021F0BD20816436E
:109C0000002306E680273F031F433F033F0B160058
:109C1000004BFEE5FF0700001E0400003E040000AC
:109C2000F8B557464E464546DE460C000903E0B5FA
:109C3000490A460F5F0031431E03DB0F760A9B463D
:109C4000530F3343C84E6500C000E40FD2006D0DC2
:109C5000A24681467F0D9C469046B74200D1B9E0AE
:109C60005B46012673409B46EE1BA34500D183E073
:109C7000002E63DD002F00D0B1E06346134300D116
:109C800023E1731E002B00D0BAE1861A6346B0426E
:109C900080410125C91A4042091A0B0200D447E14C
:109CA00049024B0A98464346002B00D189E14046C1
:109CB00000F0BCFB0300083B1F2B00DD7CE12022F1
:109CC0003000D21A4146D040994002009E400A43DB
:109CD0009D4200DD6AE15D1B6B1C1F2B00DD94E1E2
:109CE000202110003500C91A8E40DA408840DD403E
:109CF000711E8E4111000722284300250643324081
:109D0000002A09D00F233340042B05D0331DB34262
:109D1000B641764289191E000B0200D43DE26A1C4E
:109D2000914B55056D0D9A4200D119E18F4AF60805
:109D30000A40570752023743120B9BE0002E00D017
:109D4000C5E06E1C7605760D012E00DC48E1674605
:109D5000861ACB1BB042BF417F42B8461F00434624
:109D6000FF1A3B00B8461B0200D55FE137439AD18A
:109D700000220024002579E0002E00DCFAE0002F0C
:109D800000D18DE0784B9D4267D0802367461B044D
:109D90001F43BC46382E00DC52E1634613435A1E73
:109DA00093411E1886428041404209180B0200D49C
:109DB000BEE06D4B01359D4200D1D2E06B4A730885
:109DC0000A4001210E401E435108D30707221E43BB
:109DD000324095E71E00164300D045E740E7624B4E
:109DE0009D423AD0802367461B041F43BC46382E51
:109DF00000DDEBE01F2E00DC3AE133006746203B3C
:109E0000DF403B00202E05D04027BF1B6646BE40EA
:109E1000324390464646721E96413343DAE0002BA9
:109E200000D114E26346134300D168E180234E075A
:109E3000C008C9081B030643194208D06046C00881
:109E4000184204D163460100D2085E071643F300AE
:109E50009946C900720F444D11434B46DE08424BF0
:109E60004F073743CA089D4200D16EE012036D05CB
:109E7000120B6D0D00211203130B0A0D12051A436C
:109E80003B4B2D0513402B435B00E4075B0823434A
:109E9000380019003CBC90469946A246AB46F8BD36
:109EA0006346134311D0731E002B00D007E18618C0
:109EB0008642804161444042091801250B0237D592
:109EC00002257BE73E00614691463500C5E75C46CA
:109ED000002D00D0E1E00B000343F3D0731C00D150
:109EE000ACE1214B9F4200D13AE1F343382B00DD36
:109EF0006FE11F2B00DD8CE120250E00ED1AAE4036
:109F0000B0460600AA46DE40454635432E0055467B
:109F1000D940A8406346451EA8415B1A9C46304381
:109F2000161AB242924163465242991A3D00B4E673
:109F300007223240002A00D0E4E60B4BF6084F0718
:109F40003743CA089D4200D090E73B00134300D13D
:109F5000A6E180231B031A431203120B024D89E76B
:109F600015000022002785E7FF070000FFFF7FFFA5
:109F7000FFFF0F80002E00D0C7E06B1C5E05760D42
:109F8000012E00DCF0E0C84DAB4200D1B9E08518ED
:109F90000A00854289416244494251180722CE078E
:109FA0006D082E43490832401D00A9E6BF49ED1A4D
:109FB000114007223240A3E63200283882400026B2
:109FC00086E6300000F032FA203073E66346134331
:109FD0005A1E9341C61AB04280414042091A5CE6BB
:109FE0000E00674606431743002D5ED1002E00D0B9
:109FF000F3E0002F00D11EE15C46614691462CE75C
:10A00000A94FBE427BD01E00F1E610001F3DE84084
:10A01000202B03D04021CB1A9A401643731E9E4139
:10A020000722064332400021002583E7161A6346C3
:10A03000B2428041591A40420B1A98465C4632E6B9
:10A040001F2E00DDABE02027BB1B9A466346574618
:10A05000BB40994613004F46F3401F433B00574611
:10A06000BA40571EBA4113436246F240891898E637
:10A070002027BB1B9A4663465746BB4099461300B0
:10A080004F46F3401F433B005746BA40571EBA4164
:10A0900013436246F240891A9CE7834B9F425FD08C
:10A0A00080252D047342294320E7002E0CD1002F78
:10A0B00000D1D0E05C46614691467B4DCDE67A4FBB
:10A0C000BE421CD01E0065E6002F18D0C0084E0707
:10A0D00006438020C9080003014208D06346DC081B
:10A0E000044204D12100DA46D2085E071643F30089
:10A0F000994601245346C900720F11431C406A4D12
:10A10000ABE61D0000220027B4E6002D59D10B005C
:10A11000034300D1D6E6731C00D1B2E0624B9F42EC
:10A120001ED0F343382B6FDC1F2B00DD97E020257A
:10A130000E00ED1AAE40B0460600AA46DE40454687
:10A1400035432E005546A840D940451EA8418C44B1
:10A150000643B61896429241514261443D0025E6BD
:10A160003D006146914678E60B000343002D00D088
:10A1700055E6002BF5D06346134300D16DE68618F3
:10A180008642804161444042091800220B0200D4FB
:10A19000D0E6464B01351940B2E5B1465DE63300E5
:10A1A0006746203BDF403B00202E05D04027BF1BE9
:10A1B0006646BE40324390464646721E9641334341
:10A1C000EFE5394B9F42CBD080252D0473422943C4
:10A1D000A8E70843411E8841A2E6002F00D13CE6D3
:10A1E0006346861ACF1AB0429B415B42FB1A9846DF
:10A1F0001B024ED5161A6346B2429241591A524278
:10A20000891A5C4600227BE501430E00711E8E41D7
:10A210009FE71D000E00203DEE40B046202B04D0ED
:10A220004025EB1A99400843814648464346411E63
:10A230008841184374E60022002417E6161A634684
:10A24000B2429241591A5242891A3D0025E56146AF
:10A250009146154D01E680220024120379E61D0087
:10A260000E00203DEE40B046202B04D04025EB1AD6
:10A270009940084381464E464346711E8E411E4317
:10A2800067E7861896429B4161445B42C9183D00CE
:10A290008CE547463743CED007224146324049E657
:10A2A00000273A00E6E5C046FF070000FFFF7FFFFA
:10A2B00070B50C4E0D031C0349005B002D0B490DBE
:10A2C000240B5B0DB14208D0064900208B4203D11C
:10A2D00014432000441EA04170BD05430120002D01
:10A2E000FAD1F1E7FF07000030B5144D0A034B0027
:10A2F000120B5B0DC90F0024AB4211DD104CA342C1
:10A3000010DC8024640322430E4CE41A1F2C0CDD65
:10A310000D48C31ADA4013005C42002900D11C002A
:10A32000200030BD094BCC18FAE7094DE040AC469F
:10A3300063449A4013000343EEE7C046FE03000067
:10A340001D0400003304000013040000FFFFFF7F22
:10A35000EDFBFFFF70B500282DD0C317C5185D4079
:10A36000C40F280000F062F8154B1B1A5B055B0D4B
:10A370000A2815DD0B38854000222D032D0B002106
:10A3800010002D030A0D2D0B12052A430D4D1B0540
:10A390002A4013435B00E4075B082343190070BDA8
:10A3A00002002900153291400A000B21081AC5400D
:10A3B0002D032D0BE3E70024002300250022DEE718
:10A3C0001E040000FFFF0F8010B5041E25D000F012
:10A3D0002DF8144B1B1A5B055B0D0A2812DD0B3898
:10A3E000844000222403240B0021100024030A0DC2
:10A3F000240B120522430C4C1B05224013435B0027
:10A40000590810BD02002100153291400A000B21AD
:10A41000081AC4402403240BE6E70023002400228A
:10A42000E2E7C0461E040000FFFF0F801C2101234D
:10A430001B04984201D3000C10391B0A984201D327
:10A44000000A08391B09984201D30009043902A205
:10A45000105C40187047C04604030202010101016C
:10A46000000000000000000010B5040004481300C4
:10A47000002804D00A000220210000E000BF10BD27
:10A480000000000070B500260C4D0D4C641BA4109C
:10A49000A64209D1002603F02FFB0A4D0A4C641B8B
:10A4A000A410A64205D170BDB300EB589847013601
:10A4B000EEE7B300EB5898470136F2E76C02002054
:10A4C0006C0200206C02002094020020EC30006836
:10A4D00070470000044B1B681B6A002B00D1034B24
:10A4E000EC3318687047C046340000209800002004
:10A4F00010B5034B0100186800F014FB10BDC046F6
:10A500003400002010B5034B0100186800F0C0FAB9
:10A5100010BDC0463400002082B0002900D101A93E
:10A52000101E06D0002B06D013780B601078431E47
:10A53000984102B0704702204042FAE7002310B56C
:10A540009A4200D110BDCC5CC4540133F8E710B579
:10A55000884202D98B18984203D3002307E08B5C12
:10A560008354013AFBD210BDCC5CC45401339A42EF
:10A57000FAD1F8E703001218934200D1704719701E
:10A580000133F9E7F7B5016804003B290BD93C22F8
:10A59000684601F0BFFA63680099019A5B1863602E
:10A5A000002A51DB226061683B290BD93C226846B6
:10A5B00001F0B0FAA3680099019A5B18A360002A21
:10A5C00047DB6260A16817290BD91822684601F0A1
:10A5D000A1FAE3680099019A5B18E360002A3DDB69
:10A5E000A26021690B290BD90C22684601F092FA6E
:10A5F00063690099019A5B186361002A33DB226169
:10A6000065691C23AA070FD164212800FEF72CF9E5
:10A610001D23002908D13C4B9131E818FF31FEF78A
:10A6200023F94B424B411C33E2681D27002A45DDCC
:10A6300003261C272269E168012A43D0334D90008C
:10A640004059814241DC3CE03C32013B2260636086
:10A65000A9E73C32013B6260A360B3E71832013BDB
:10A66000A260E360BDE70C32013B22616361C7E792
:10A670002269013A2261013217D10B230322656955
:10A680002361681E6061113310420ED16421FEF710
:10A69000EBF83B00002908D11D4B9131E818FF3140
:10A6A000FEF7E2F84B424B411C3321691A000129A5
:10A6B00002D0164A89008A58B618E660E668002E6D
:10A6C000D6DDF7BD8B42FCDA1800091A0132E160D1
:10A6D00022610C2AAED1002365692361681C606188
:10A6E0003B003042A6D16421FEF7BEF81D230029AD
:10A6F000A0D1084B9131E818FF31FEF7B5F84B4275
:10A700004B411C3396E7C0466C07000080E2000016
:10A710006B0700006D070000F0B58BB0040002F07D
:10A72000B9F807002000FFF72DFF3C236268A168FD
:10A73000534322689B18E12212014A439B1800935D
:10A74000E268DB1701932369501EB54A99008A58C5
:10A750008218049262690392012B14DD13009B0797
:10A7600011D164211000FEF77FF8002908D1039B66
:10A77000AC4A9131FF319818FEF776F8002902D1E2
:10A78000049B01330493049BA749E361039BA74AFD
:10A790005B18934200D974E1039B462B00DC88E0F0
:10A7A000C8264625760003231D4200D07FE06421A1
:10A7B0002800FEF759F8B7235B00002908D1994B10
:10A7C0003100E818FEF750F84B424B416E33FF332F
:10A7D000049A0135D3180493039BAB42E3D1049A46
:10A7E000934B53431800D917009A019B12184B4101
:10A7F0000092019300F0FAFF00F0FAFF8D4B1D6804
:10A80000002D4CD06369874A9818236A05930893F2
:10A81000002B01DD012308937B68834200D089E08F
:10A82000B86CF96C3B6D02000993099B0693DB172A
:10A830000793BB6A1D00DE179C460B00521BB341F9
:10A840001E00019B15009E420EDC02D1009B9D4222
:10A850000AD8069A079B801A9941019B99426EDC9F
:10A8600002D1009B98426AD8069807993A6A7B6A97
:10A87000121A8B413968002963D001998B420ADC96
:10A8800002D100998A4206D8019B9E4260DC02D127
:10A89000009B9D425CD8059B0025002B5CDABB6ABF
:10A8A0001E00DF17009A019BB6185F41A6E06E23D9
:10A8B0008DE7039B462B92D0C8264525760016E0EF
:10A8C000002B30D164212800FDF7CEFFB7235B00B9
:10A8D000002908D1534B3100E818FDF7C5FF4B4262
:10A8E0004B416E33FF33049A013DD31A0493032383
:10A8F000039A2B40AA42E3DB002B16D164211000FF
:10A90000FDF7B2FF002912D1039B464A91319818F6
:10A91000FF31FDF7A9FF4B4259416E31FF31049BD6
:10A920005B1A04935BE76E23DCE76E21F6E7B72141
:10A930004900F4E700F0AAFE002800D070E7089D67
:10A9400051E001998B429FDC02D100998A429BD849
:10A95000059B0125002B49DB089E6E40012E42D14C
:10A960006346099A9B1A002D00D15B4218002268A9
:10A97000D917D2182260009A019B12184B410092FD
:10A980000193E36820000593FFF7FCFDE368059A57
:10A990009B1A28D0012B20DC5A1C00DB1E00049BD4
:10A9A000E2699B1904930323B61847D5039A501EF6
:10A9B000184215D16421FDF757FF00292DD11E4AF9
:10A9C000039B9446913163441800FF31FDF74CFF1F
:10A9D0004B4259416D31FF3104E001267642DEE7FA
:10A9E000B6214900E161012D00D058E73B6D0125FA
:10A9F0001E00DF17009A019BB6185F4100F0F7FEBA
:10AA00000498256204300721FDF72EFF002936DB6C
:10AA1000A161300039000BB0F0BD6E21DBE7C0460C
:10AA2000B0E200006C07000010270000204E00007C
:10AA300080510100101000206B070000039A1A4299
:10AA400016D164211000FDF70FFF002912D10F4A23
:10AA5000039B9446913163441800FF31FDF704FFD6
:10AA60004B4259416E31FF318E4206DAE661BAE758
:10AA70006E21F8E7B7214900F6E7761AF6E70731C5
:10AA8000C6E701267642F717C3E7C0466C07000009
:10AA900070B50500002910D00C1F2368002B00DAC8
:10AAA000E418280001F011FF1D4A1368002B05D19E
:10AAB00063601460280001F009FF70BDA34209D94A
:10AAC000216860188342F3D118685B6841182160DF
:10AAD000EEE713005A68002A01D0A242F9D919689A
:10AAE0005818A0420BD120680918581819608242E2
:10AAF000E0D110685268411819605A60DAE7A04244
:10AB000002D90C232B60D5E721686018824203D15B
:10AB1000106852684118216062605C60CAE7C046F4
:10AB2000EC0F0020032370B5CD1C9D4308350600B3
:10AB30000C2D1ED20C25A9421DD8300001F0C5FEF7
:10AB4000254A14682100002919D1244C2368002BC0
:10AB500003D1300000F0ACFC20602900300000F090
:10AB6000A7FC431C2BD10C233000336001F0AEFE58
:10AB700003E0002DDFDA0C233360002070BD0B688A
:10AB80005B1B19D40B2B03D90B60CC18256003E099
:10AB90004B688C420DD11360300001F097FE20000D
:10ABA00007220B30231D9043C31AE7D05A42E250CC
:10ABB000E4E763600C00EFE70C004968C3E7032398
:10ABC000C41C9C43A042E1D0211A300000F070FC6C
:10ABD000431CDBD1C7E7C046EC0F0020F00F00207C
:10ABE000F0B58BB014001D1E129953DA8024240690
:10ABF0001B191D0014002D230B702023149E03220B
:10AC00009E43462E07D03300453B59424B41109995
:10AC1000013ACB18109309AB049308AB0393139B31
:10AC200000920293109B220001932B0001F010F878
:10AC30000700472E02D1119BDB0724D5109BFB1880
:10AC40000793462E14D13B78302B0CD100220023E1
:10AC500020002900FDF71EFE002804D10123109AD0
:10AC60009B1A139A1360139B079A1B68D3180793B8
:10AC70000022002320002900FDF70CFE30220028CE
:10AC80000DD0079B09933800099B159ADB1B1360B5
:10AC90000BB0F0BD0023AFE7591C09911A70099B56
:10ACA00007998B42F8D3EEE7F0B5831C85B001938A
:10ACB00006000C0002702B23002901DA2D234C42E0
:10ACC0007370092C22DD02ABDD1D20000A21FDF787
:10ACD000CBFD6F1E3031397020000A21FDF7DEFCFC
:10ACE000040009280BDC023D3034019B2C7002AAC1
:10ACF00007321800AA4204D8801B05B0F0BD3D0001
:10AD0000E3E72A7801351A700133F0E73023E418BD
:10AD1000B370301DF470EFE7F0B595B00C000A92F7
:10AD20000B931A9D099001F0B9FD036818000C936C
:10AD300000F002FC0023129323680E900D930D99EE
:10AD4000277E2B680722C90545D59B1893431A0017
:10AD500008322A601A685B68A264E3640122E56C29
:10AD6000A66C6B005B080F935242AC4B30000F99FE
:10AD7000FFF79EFA002830D10122A84B5242300042
:10AD80000F99FDF797FD002827D1002200233000FE
:10AD90002900FDF785FD002803D023002D22433331
:10ADA0001A709F4D472F00D89E4D032300260D9A01
:10ADB000236101339A4322600B9B13AA0093210065
:10ADC0000A9B099800F0F4F9431C00D093E001209D
:10ADD000404215B0F0BD0733B8E732002B00300019
:10ADE0002900FFF765FA002804D08F4D472FDCD8E3
:10ADF0008E4DDAE780230D996268DB000B43511C0E
:10AE000043D10732626012AA0021059211AA03926F
:10AE1000232223600691019308A9636852180292C5
:10AE2000009332002B0004970998FFF7D9FE2023E6
:10AE30003A0005009A43472A07D1119BDA1C02DB2E
:10AE40006268934245DD023FFFB21199652F25D814
:10AE5000200001393A0050301191FFF725FF129A76
:10AE6000060013182361012A02DC2268D20701D5EB
:10AE700001332361232308AA9B181B78002B9BD046
:10AE800023002D2243331A7096E7672F00D176E115
:10AE9000472FB8D1002AB6D10122B3E7662F19D1C6
:10AEA000636800290CDD2161002B02D12268D207E2
:10AEB00002D501335B182361119B0026A365D9E7F6
:10AEC000002B03D101222168114200D09A1C22617B
:10AED000F2E76727119B129A934205DB22682361F0
:10AEE000D207E9D50133E6E70121002B01DC49183F
:10AEF000C91A5218EBE72268530508D423692A00BF
:10AF00000A9909980B9DA847431C29D15FE7652F33
:10AF100000D8E0E0A06CE16C00220023FDF7BAFC51
:10AF2000002834D00123424A0A9909980B9DA8476A
:10AF3000431C00D14BE7119B129A934202DB23681A
:10AF4000DB070DD50B9D0E9B0C9A0A990998A84713
:10AF50000025431C00D13AE7129B013BAB420ADCBF
:10AF600023689B0700D508E1139BE068984200DB4B
:10AF70002FE718002DE7220001231A320A990998B9
:10AF80000B9EB047431C00D121E70135E4E7119B3C
:10AF9000002B2DDC0123264A0A9909980B9EB04705
:10AFA000431C00D113E7119B002B05D1129B002BF2
:10AFB00002D12368DB07D3D50B9E0E9B0C9A0A990E
:10AFC0000998B0470026431C00D100E7119B5B4263
:10AFD000B34201DC129B92E7220001231A320A9944
:10AFE00009980B9FB847431C00D1F0E60136EDE706
:10AFF000A36D129F9F4200DD1F00002F08DD3B0064
:10B000002A000A9909980B9EB047431C00D1DEE63E
:10B0100000230D93FB43DB170F9318E0FFFFEF7F37
:10B02000E4E20000E0E20000ECE20000E8E2000000
:10B0300052E60000220001231A320A9909980B9E59
:10B04000B047431C00D1C2E60D9B01330D930F9B0B
:10B05000A66D0D9A3B40F31A9342EBDC119B129ABA
:10B06000AD19934210DB2368DB070DD4129F119BAF
:10B07000BE1BFF1AB74200DD3700002F0DDCFE4378
:10B08000F31700250C931CE00E9B0C9A0A99099863
:10B090000B9FB847431CE9D199E63B002A000A9967
:10B0A00009980B9DA847431CE9D190E62200012393
:10B0B0001A320A9909980B9EB047431C00D186E6C4
:10B0C0000135119A129B0C999B1A3A000A409B1A5F
:10B0D000AB42EBDC44E7129B012B02DC01231A425A
:10B0E00032D001232A000A9909980B9FB847431CC4
:10B0F00000D16CE60E9B0C9A0A9909980B9F0135BA
:10B10000B847431C00D162E6A06CE16C129B0022A0
:10B110005F1E0023FDF7BEFB3B00002814D0002576
:10B120000AE0220001231A320A9909980B9FB847B6
:10B13000431C00D14BE60135129B013BAB42F0DCD6
:10B14000220033005032DBE62A000A9909980B9D51
:10B15000A847431CF4D13AE62200012319320A9988
:10B1600009980B9EB047431C00D130E60135E368D7
:10B17000139A9B1AAB42EFDCF6E60025F7E7002AAC
:10B1800000D189E60021069112A9059111A9039128
:10B19000232108A809182360019300922B0004972B
:10B1A000029132000998FFF71BFD050045E6C046F5
:10B1B000F7B5150001938A680B6900900C00934263
:10B1C00000DA130022002B6043321278002A01D0EB
:10B1D00001332B6023689B0602D52B6802332B605A
:10B1E000062723681F4027D0230043331B785A1EAD
:10B1F00093412268920630D422000199433200988C
:10B20000089EB047431C25D0062320682A68E168C1
:10B2100003400025042B03D18D1AEB43DB171D409F
:10B22000A3682269934201DD9B1AED180027BD42F5
:10B2300020D1002010E00137E3682A689B1ABB4246
:10B24000D2DD22000123193201990098089EB047EF
:10B25000431CF0D101204042FEBD3020E1184331B3
:10B26000087021005A1C45310978A2184332023374
:10B270001170C1E7220001231A3201990098089E3B
:10B28000B047431CE6D00137D1E70000F0B589B0E4
:10B2900004920A0043320593039002920A7E0C0046
:10B2A0000E9B6E2A00D186E01FD8632A33D008D8BF
:10B2B000002A00D18CE0582A4DD0250042352A7052
:10B2C00030E0642A01D0692AF7D1196825680A1D7F
:10B2D000280629D508681A60002803DA2D23029A67
:10B2E000404213706B4E0A274FE0732A74D008D87F
:10B2F0006F2A1FD0702AE0D1202209680A432260F9
:10B3000003E0752A16D0782AD7D122007821453259
:10B310001170614E22E025001A684235111D196036
:10B3200013682B70012365E008681A606906D3D59D
:10B3300000B2D1E719682568081D186008682E0654
:10B3400005D5544E08276F2A1BD00A2719E06D0631
:10B35000F7D580B2F5E745314E4E0A70186822687D
:10B36000011D00681960150621D5D30702D52023D9
:10B370001A4322601027002803D1202322689A4311
:10B3800022602300002243331A706368A360002BFD
:10B3900058DB0422216891432160002854D1029D8A
:10B3A000002B5AD02500337842352B7055E05506D6
:10B3B000DBD580B2D9E71A680D68101D496918609D
:10B3C00013682E0601D5196002E06D06FBD51980C1
:10B3D0000023029D23614FE01A68111D1960156852
:10B3E00000216268280001F065FA002801D0401BA6
:10B3F0006060636823610023029A13703CE0236954
:10B400002A0004990398059DA847431C3ED0236851
:10B410009B0715D4079BE068984239DA180037E09B
:10B4200022000123193204990398059EB047431C5A
:10B430002CD00135E368079A9B1AAB42F0DCE9E7B0
:10B440000025F7E70028ADD0029D3900FDF722F96D
:10B45000735C013D2B700028F7D1082F09D12368B8
:10B46000DB0706D563682269934202DC3023013D85
:10B470002B70029B5B1B2361059B07AA0093210095
:10B48000049B0398FFF794FE431CB8D1012040426F
:10B4900009B0F0BDF0E2000001E3000010B5034B7D
:10B4A0000A000100186801F007FD10BD34000020FB
:10B4B000002370B5064C05000800236002F00EFB67
:10B4C000431C03D12368002B00D02B6070BDC04605
:10B4D000081100200EB400B50B499CB01DAB0290C2
:10B4E0000690079104910948094904CB0591006829
:10B4F00002A9019301F068FD0023029A13701CB0A9
:10B5000008BC03B01847C046FFFFFF7F340000208F
:10B510000802FFFF02780B78002A03D001300131C6
:10B520009A42F7D0D01A704703000A7801311A7096
:10B530000133002AF9D170470023C25C0133002A8D
:10B54000FBD1581E7047002330B59A420AD0013A09
:10B55000C45CCD5CAC4204D1934202D00133002CD8
:10B56000F6D1631B180030BDF0B51F000E0087B088
:10B570000590019102920C983478FEF7A7FF0822FB
:10B5800000194378751C134036D12D2C36D1B51CCB
:10B5900074780126002F62D0102F09D1302C07D1EA
:10B5A00020222B789343582B54D110276C780235E6
:10B5B0002D4B3900F31818000393FDF76BF8049135
:10B5C00001210023494202008C4618002100303935
:10B5D00009291AD80C00A74223DD591C09D063465B
:10B5E000824206D302D10499A14202DB01237843AF
:10B5F00020182C780135E9E72E00BCE72B2C01D070
:10B600001E00C7E7B51C7478FAE7210041391929F3
:10B6100001D8373CDFE721006139192901D8573CAF
:10B62000D9E75A1C08D1059A23331360029B03986B
:10B63000002B09D107B0F0BD002E00D04042029A85
:10B64000002AF7D0002B01D06B1E0193029B019AB8
:10B650001A60EFE73024002FAAD10827A8E7302C82
:10B660009ED00A27A4E7C046FFFFFF7F13B5054C15
:10B670002468246A002C00D1034C0094FFF774FF67
:10B6800016BDC0463400002098000020F0B589B0F7
:10B69000040001F0FFF84E4B060000209C425FDDE5
:10B6A0006E2564214B4BFF35E01845434A4B7460CF
:10B6B000E0184A4B80102D184942E018FCF7EEFFC5
:10B6C000C821474B2D184900E018FCF7E7FF64211B
:10B6D0002B1820000093FDF7C7F80191C821200026
:10B6E0004900FDF7C1F80A0053425A41330058336C
:10B6F0000793032335001C400291049208350594FA
:10B700002B78EF684A2B2DD1009BDC19059B002B71
:10B7100002D1019B002B03D10021029B8B4203D15C
:10B7200001213B2F00DC00216418013C2D492B69CD
:10B730004C43E4182B6AE418AC61079BE417EC61F6
:10B740002835AB42DCD1F16C726A0123914205DCF1
:10B7500003D1B26C316A8A4200D8002301203360E1
:10B7600009B0F0BD442B02D1009BDC19DEE7059B3C
:10B77000049A002B03D1019B002B00D0012230231F
:10B7800053430693184B00219C466868009C069A18
:10B7900001318B009B186246043BD35803938842C7
:10B7A00010DC201D0721FDF75FF8791A00D507315D
:10B7B000AB685A1E072353435918039B994204DA76
:10B7C0006418B3E7039BE418E1E70739F5E7C046DF
:10B7D000B10700004EF8FFFF4FF8FFFF93F8FFFF9F
:10B7E000BFF9FFFF80510100BCE4000070477047C3
:10B7F00010B5024B186800F003F810BD34000020AB
:10B80000F0B58DB0070001F045F8AF4906003800EB
:10B8100001F03AF8AD4D041E0DD1AD4BAD4A1860A4
:10B82000AD4B1860AD4B28681A605A60FEF76AFE8F
:10B830002C600DB0F0BD2968002959D12868FEF7A9
:10B8400061FE2000FFF778FE411C3800FFF76AF91F
:10B850002860002851D12378A1493A3B5A425341EC
:10B86000E418A04A0AAB200001F0ACFC0028E0DD9F
:10B870000A9BE41823782D2B43D12E3B01340493EB
:10B88000162702ABFF18002308AD3B802B800AABC4
:10B89000039302950193009707AA9349200001F0B2
:10B8A00091FC0028C5DD3C233A88904F53432A88F9
:10B8B0008A4D9B1802AA918AE12212014A439B18E1
:10B8C000049A87495A43874BB2622B600A9B3A001D
:10B8D000E41820000AAB01F075FC002818DC2B6886
:10B8E000B26A6B607A4B1A6000227B4B1A60A0E749
:10B8F000FFF710FE00289CD0A0E72100FFF714FE00
:10B90000A9E701222B3B04925A425341E418B7E7BE
:10B910000A9B6F60E41823782D2B00D08DE02E3B1E
:10B92000013404931627002302AABF1807AD13831E
:10B930002B803B8008AA0A930AAB029203930193DF
:10B9400000972A006849200001F03CFC002800DD37
:10B950007AE0B36A664A9B1833650A9B3700E4189D
:10B9600000230837049323782C3B5A425341E418B0
:10B9700025784D2D00D078E01E2202A9521802929F
:10B9800009AA00921A220AAB52180393019359494B
:10B99000200001F017FC032800D04AE702AB598BC6
:10B9A0004B1E0B2B00D944E702AB9A8B531E042B82
:10B9B00000D93EE702ABDB8B062B00D939E73D709F
:10B9C0007960BA60FB600A9BE518022307AA13801E
:10B9D000002302A908ACCB8223800A932B782F2B5B
:10B9E0000BD1162102A809180AAB00910393029407
:10B9F00001934149280001F0E5FB02ABDA8A3C23C0
:10BA0000534322889B1807AA1188E12212014A4356
:10BA10009B183B610A9B2837EC18049B012B22D111
:10BA20007068FFF733FEB26A294B1A60336D9B1AB8
:10BA30005A1E9341284A1360FBE601222B3B0492D5
:10BA40005A425341E4186DE73C233A88298853430E
:10BA500002AA128B9B18E12212014A439B18049AF6
:10BA60005A43130078E701237CE7442305934A2DCA
:10BA700001D1013405950A220BA9200001F060FCD8
:10BA80001E2302AA0B9D9B181880A54216D1049B69
:10BA9000002B08D14D3333720323F360013B336134
:10BAA000049B736191E733004D2230331A700B23EE
:10BAB00073630A3BB3630023F36386E76B461B7D26
:10BAC00080B23B70F86080E712E300000C100020A9
:10BAD0001410002015E300001010002004020020C4
:10BAE00019E30000FF0F00203CE30000F40F0020EA
:10BAF000F0F1FFFF28E300003BE300000B1E04D041
:10BB0000FF2A04D98A2303608B3B180070470A7010
:10BB10000123FAE770B50E00040011003000150093
:10BB2000FCF7A2FE002E07DB002901DA0130491BD9
:10BB300020606160200070BD0029F9DD01384919DD
:10BB4000F6E7F0B503690C6989B007000591002696
:10BB5000A34265DB0B00013C1433A50003935B1982
:10BB600004930300143302935D19049B28681B6837
:10BB7000591C0193FCF708FD0190B04229D0039BAA
:10BB800002989C460696624608CA9446019A99B263
:10BB900051431B0C534389190A0C9B1807931E0C25
:10BBA000036889B29AB2069BD2180368521A190C1C
:10BBB0006B469B8BCB1A11145B18191492B21B04A1
:10BBC0001A43049B069104C06345DCD22B68002B0A
:10BBD0002DD00599380001F08FF800281FDB0025D3
:10BBE000019B0298013303990193026808C992B23C
:10BBF00055199AB2AA1A05681B0C2D0CEB1A1514CC
:10BC00005B191D1492B21B04134308C0049B8B42A2
:10BC1000EBD2029AA300D3181A68002A11D0019E11
:10BC2000300009B0F0BD2B68002B04D1013C029B11
:10BC3000043DAB42F7D33C61CBE71A68002A04D13C
:10BC4000013C029A043B9A42F7D33C61E7E70000CB
:10BC5000F0B516001F00446A9BB00290239D069623
:10BC60000797002C08D11020FEF742FC029B586277
:10BC7000446084600460C460029B5B6A19680029A8
:10BC80000BD05A68012393404A608B60029800F001
:10BC900056FE0022029B5B6A1A60002F20DA012305
:10BCA0002B607B005B080793079CB24B2200179325
:10BCB0001A409A4217D1B04B229A1360069B002B70
:10BCC00003D1240301D100F087FDAC4B249A0893E3
:10BCD000002A02D0AA4B249A136008981BB0F0BD2A
:10BCE00000232B60E0E7069E079F00220023300020
:10BCF0003900FCF7CFFD051E0BD00123229A1360FB
:10BD0000A04B249A0893002AE7D09F4A24990A60FE
:10BD1000E3E718AB019319AB009332003B000298A4
:10BD200001F068F8630003905B0D74D03A03974C00
:10BD3000120B14432100964A300016959E180022DB
:10BD4000944BFDF76DFF944A944BFDF7F7FC944A32
:10BD5000944BFCF7CDFD040030000D00FEF7FAFA1D
:10BD6000914A924BFDF7EAFC02000B0020002900EB
:10BD7000FCF7BEFD04000D00FEF7B6FA0022070036
:10BD8000002320002900FCF78BFD002809D0380093
:10BD9000FEF7E0FA2B002200FCF77CFD43425841FD
:10BDA0003F1A01231493162F0DD88149FB00C9189F
:10BDB00008684968069A079BFCF786FD002846D06C
:10BDC0000023013F1493189B9E1B00230A9333000A
:10BDD000013B0B9304D501239B1B0A9300230B9378
:10BDE000002F36DB0B9B1197DB190B930023049379
:10BDF000209B0124092B00D984E0052B02DD0024BF
:10BE0000043B2093209B981E032800D984E0FCF774
:10BE1000B1FB7577286A189B199A9E18654BF21822
:10BE2000202A0FDD40239B1A9C40634B0698F31891
:10BE3000D8402043FEF7C8FA0123604C013E09199F
:10BE400016937CE7202306989B1A9840F2E71490FB
:10BE5000B9E70A9BDB1B0A937B42049300231193EF
:10BE6000C6E701230D93219B002B59DD0C93099309
:10BE7000029A556A00226A60043210001430696820
:10BE8000984252D9029800F022FD029B28605B6A1A
:10BE90001B680893099B0E2B00D90AE1002C00D1E6
:10BEA00007E1069B079C12931394002F00DC89E0A6
:10BEB0000F213A003E4B0A40D2009B181D685E6875
:10BEC00002233C110E93E3060BD53D4B0C401A6A3E
:10BED0005B6A12981399FDF727F8032306900791E0
:10BEE0000E9300233AE001230D93219BFB180C9342
:10BEF00001330993002BBBDC0123B9E70023B1E731
:10BF00000023F1E700230D942093013B00220C93C2
:10BF1000099313332192ABE701230D93023BF5E71D
:10BF200001230C9309931A00F4E701316960520070
:10BF3000A3E701231C420ED00E9B214A01330E932E
:10BF4000109B2800DB009B1831001A685B68FDF726
:10BF5000F5FB05000E00109B641001331093002CBC
:10BF6000E7D1069807992A003300FCF7DDFF069019
:10BF7000079142E00000F07F0F27000058E4000026
:10BF80005BE4000052E6000053E600000000F03FD2
:10BF900001FCFFFF0000F83F61436F63A787D23FBA
:10BFA000B3C8608B288AC63FFB799F501344D33FA8
:10BFB00048E500003204000012040000000010FEFA
:10BFC00020E5000002230E93002F16D0129813993B
:10BFD0007C420D332340CE4ADB00D3181A685B68DD
:10BFE000FDF7ACFB002301261D00069007912411EC
:10BFF000002C00D08CE0002BB9D1149B002B00D179
:10C0000096E0069C079D0022C24B20002900FCF709
:10C0100047FC002800D18BE0099B002B00D187E072
:10C020000C9B002B41DDBC4B002220002900FDF7BA
:10C0300085FB0E9B0690079101330E930C9B7E1E91
:10C040000E981093FEF786F9069A079BFDF776FB8C
:10C050000022B24BFCF74CFCB14A0E900F910E9CA3
:10C060000F9D94460F9B634415931D00109B002B5E
:10C0700061D1069807990022AA4BFDF7D1FD220055
:10C08000159B06900791FCF71FFC002800D0A8E242
:10C09000A5480F99844661440B0006980799220031
:10C0A000FCF7FEFB002800D095E2129B139C069340
:10C0B0000794199B002B00DA5CE10E2F00DD59E19B
:10C0C000934BFA009B185C681B6804930594219BB2
:10C0D000002B00DBD8E0099B002B00DDD4E000D072
:10C0E0007DE20498059900228E4BFDF727FB069A06
:10C0F000079BFCF7F3FB099B04931E00002800D06C
:10C100004FE2089B089A5D1C3123013713704BE204
:10C1100034420AD00E9B854A01330E93EB009B18E4
:10C120001A685B68FDF70AFB3300641001355FE7AE
:10C130003E00099B84E7109B0D995A1E744BD20058
:10C140009B181A685B68002949D000207849FCF7E1
:10C15000EBFE2B002200FDF763FD089B0E900F9174
:10C16000159306980799FEF7BFF80400FEF7F2F85A
:10C1700002000B0006980799FDF752FD159B30341D
:10C180005D1C1C700E9A0F9B06900791FCF788FBB4
:10C1900000286CD1069A079B00205E49FDF740FD00
:10C1A0000E9A0F9BFCF77CFB002800D0C3E0089B95
:10C1B000109AEB1A9A4200DC77E70E980F9900224A
:10C1C000554BFDF7BBFA00220E900F910698079988
:10C1D000514BFDF7B3FA159506900791C1E7200082
:10C1E0002900FDF7ABFA089C109A230094460E90A4
:10C1F0000F916344159306980799FEF775F80500AB
:10C20000FEF7A8F80B00020006980799FDF708FD55
:10C210003035159B2570013406900791A3422AD131
:10C220000E980F99089A109B9446634400221D00B3
:10C230003F4BFCF75DFB02000B0006980799FCF7EB
:10C2400043FB002800D076E00E9A0F9B002038496F
:10C25000FDF7E6FC02000B0006980799FCF720FBAF
:10C26000002800D121E76B1E1A78302A01D0370050
:10C270003FE01D00F7E7069807990022264BFDF7DF
:10C280005DFA06900791B6E7089E049A059B06980A
:10C290000799FCF749FEFEF727F80400FEF75AF865
:10C2A000049A059BFDF74AFA02000B0006980799CD
:10C2B000FDF7B6FC230030333370099A089B751CD8
:10C2C000EB1A9A4248D102000B00FCF711FB049ACA
:10C2D000059B06900791FCF7F7FA00282AD1049AEB
:10C2E000059B06980799FCF7D5FA002801D0E307CB
:10C2F00020D40399029800F022FB00232B70229B8C
:10C3000001371F60249B002B00D1E6E41D60E4E4AC
:10C3100048E500000000F03F0000244000001C4001
:10C320000000C0FC000014400000C07C20E50000BC
:10C330000000E03F3E006B1E1A78392A06D1089AA9
:10C340009A4207D130231370130001361A78013254
:10C350001A708CE71D00EEE70022A44BFDF7EEF902
:10C3600000220023069007912E00FCF793FA002884
:10C370008BD0BEE70D9A002A00D1DAE0209A012A7C
:10C3800000DDBDE0169A002A00D1B5E0984A9B185E
:10C39000049D0A9C0A9A0121D2180A920B9A0298CB
:10C3A000D3180B9300F06BFB0600002C0EDD0B9BEB
:10C3B000002B0BDD0B9A2300944200DD13000A9A38
:10C3C000E41AD21A0A920B9AD31A0B93049B002BED
:10C3D0001FD00D9B002B00D1AFE0002D11D03100FC
:10C3E0002A00029800F0E4FB039A0100060002987C
:10C3F00000F04EFB03991090029800F0A0FA109BF9
:10C400000393049B5A1B04D00399029800F0D0FBBD
:10C4100003900121029800F032FB119B0490002B45
:10C4200000D1E3E11A000100029800F0C1FB209B5B
:10C430000490012B00DD82E00025069BAB420ED16B
:10C44000079B1B03AB420AD1179B079A134206D0E6
:10C450000A9B013501330A930B9B01330B93119B0C
:10C460000120002B6CD10B9B18181F2318407ED085
:10C4700001331B1A042B70DD1C23181A0A9B241885
:10C480001B180A930B9B1B180B930A9B002B05DDB3
:10C490001A000399029800F0DDFB03900B9B002B20
:10C4A00005DD1A000499029800F0D4FB0490149B57
:10C4B000002B5ED00499039800F01EFC002858DA87
:10C4C00000230A220399029800F052FA0D9B013FC3
:10C4D0000390002B00D190E1002331000A22029842
:10C4E00000F046FA0C9B0600002B00DD88E0209B44
:10C4F000022B00DC84E044E03623189A9B1A47E7BD
:10C50000099B5D1E049BAB4208DB5D1B099B002B56
:10C510000CDA0A9B099A9C1A00233BE7049B0495BA
:10C52000EA1A119B00259B181193EFE70A9C099BBF
:10C5300030E7049D0A9C0D9E37E7049A64E70025C6
:10C54000049B049A1B69109303339B00D31858680B
:10C5500000F04CFA2023181A85E7042B95D00A9A8C
:10C560001C33D2180A920B9AE418D3188CE70300F4
:10C57000F5E7099B002B3DDC209B022B3ADD099B54
:10C580000C930C9B002B0CD104990522029800F00F
:10C59000EFF904900100039800F0AEFB002800DDE5
:10C5A000AFE5219B089DDF4300230993049902987E
:10C5B00000F0C5F9002E00D19BE6099B002B05D0A9
:10C5C000B34203D01900029800F0B9F93100029883
:10C5D00000F0B5F98DE6109B04931E00E1E70023FF
:10C5E000FAE7109B370004931E008AE50000244000
:10C5F000330400000D9B002B00D1B2E0099B0C938B
:10C60000002C05DD31002200029800F023FB06001B
:10C610003000002D11D07168029800F058F93100F7
:10C62000040033690C319A1C92000C30FDF786FF30
:10C6300001222100029800F00DFB09960600089BDC
:10C640000A9304990398FFF77CFA09990D90040066
:10C65000039800F051FB320010900499029800F00A
:10C6600065FB01230B93C36830340500002B04D114
:10C670000100039800F040FB0B902900029800F0A5
:10C680005EF90B9B209A13430ED1069A0133134295
:10C690000AD1392C26D0109B002B01DD0D9C3134A2
:10C6A0000A9B5D1C1C7081E7109B002B07DB1D00A3
:10C6B000209B1D4322D10123069A13421ED10B9BBE
:10C6C000002BEDDD03990122029800F0C3FA0499D2
:10C6D000039000F011FB002802DCE1D1E307DFD575
:10C6E000392CDBD10A9B0A9A5D1C392313706B1E0F
:10C6F0001A78392A67D001321A7057E70A9B5D1CF5
:10C700000B9B002B04DD392CECD001340A9BC9E7CC
:10C710000A9B0C9A1C70089BEB1A93423ED0002394
:10C720000A220399029800F023F9099B0390B3426F
:10C7300009D100230A220999029800F019F90990F9
:10C7400006000A957DE7099900230A22029800F065
:10C750000FF9002309900A223100029800F008F92D
:10C76000EEE7099B0C93089B069304990398FFF747
:10C77000E8F9069B30305D1C18700C9A089B040089
:10C78000EB1A9A4208DD00230A220399029800F06E
:10C79000EFF806950390E8E7002309930399012237
:10C7A000029800F057FA0499039000F0A5FA0028C7
:10C7B0009DDC01D1E3079AD46B1E1A78302A00D091
:10C7C000F4E61D00F8E7089A9A4203D131230137B5
:10C7D0001370EBE61D008AE70B4B249A08930B4B72
:10C7E000002A01D0FFF777FAFFF777FA209B012B99
:10C7F00000DC21E6119D012035E60C9B002BB2DC0C
:10C80000209B022BAFDDBCE64FE4000057E40000A4
:10C81000F0B50E0085B00700039200F0A5FD194C9D
:10C8200033002568002D06D1380000F09EFD002061
:10C8300005B0F0BD01331A78002A1FD03D2AF9D186
:10C84000F2E7043528680028EED0019A3100FEF79F
:10C850007AFE0028F5D1019A2B689446634402932E
:10C860001B783D2BEDD123683800ED1A039BAD10EA
:10C870001D6000F07AFD02980130D9E79B1B0193FF
:10C88000E0E7C0466802002007B501AAFFF7C0FF35
:10C890000EBD00000048704710020020034B1B68CB
:10C8A000186A002800D10248F03070473400002098
:10C8B00098000020C9B28218904201D10020704730
:10C8C00003788B42FBD00130F6E77047704770B5B4
:10C8D000466A04000D00002E07D11020FDF708FE67
:10C8E0006062466086600660C660666AF368002B18
:10C8F00013D0636AAA00DB689B181868002818D157
:10C9000001210E00AE40721D9200200000F0C6FA18
:10C9100000280CD0456086600DE021220421200013
:10C9200000F0BCFA636AF060DB68002BE1D1002004
:10C9300070BD02681A6000230361C360F8E770B538
:10C94000446A06000D00002C07D11020FDF7D0FD31
:10C950007062446084600460C460002D07D0736A14
:10C960006A68DB6892009B181A682A601D6070BDB7
:10C97000F7B51E0014239C4607000C0000200D692B
:10C980008C4463461B68013099B263461B6851436F
:10C990001B0C534389190E0C9B1989B21E0C1B04E6
:10C9A0005B18614608C18C468542EADC002E1BD02C
:10C9B000A368AB4212DC63683800591CFFF787FF9D
:10C9C0002100236901909A1C92000C310C30FDF774
:10C9D000B5FD21003800FFF7B2FF019C2B1D9B0025
:10C9E000E31801355E6025612000FEBD0300020CE6
:10C9F0000020824201D11B0410301A0E01D10830F0
:10CA00001B021A0F01D104301B019A0F01D1023011
:10CA10009B00002B03DB01305B0000D4202070471B
:10CA20000722036810B501001A400DD00124002030
:10CA3000234205D10230034203D0E34020000B60C3
:10CA400010BD9B080B60FBE79CB21000002C01D1CD
:10CA500010201B0CDAB2002A01D108301B0A1A0779
:10CA600001D104301B099A0701D102309B08DA0773
:10CA7000E8D45B0801D00130E4E72020E0E710B5FE
:10CA80000C000121FFF723FF01234461036110BD66
:10CA9000F0B50B691400126989B00D00934201DAF8
:10CAA00025000C002F6926696968BB190293AB68E1
:10CAB000BA19934200DA0131FFF709FF0200BB19EE
:10CAC00014329B00D3189C46002113000490634548
:10CAD0001DD31435BF00EB191434B6000593A31908
:10CAE000039501940793079B0199994211D3029BE7
:10CAF000002B06DD04235B429C4463461B68002B2D
:10CB000051D0049B029A18001A6109B0F0BD02C30B
:10CB1000DDE7019B1B6898B200281CD01500002699
:10CB2000039F02CF2C688BB24343090C4143A4B24C
:10CB30001B199B190E0029680695090C71181E0C0B
:10CB400089190E0C9BB209040B4308C5059BBB4217
:10CB5000E7D8069B5E60019B1B681D0C1ED0100071
:10CB600000271368039E3168046889B26943240C66
:10CB70000919C9190F049BB23B43036080CE436877
:10CB80003F0C6F439BB2FB18090C5B18059906908C
:10CB90001F0C0430B142E6D806994B60019B043269
:10CBA000043301939FE7029B013B02939FE7000040
:10CBB0000323F7B5134005000E001400002B08D026
:10CBC0002249013B9A00525800233100FFF7D0FE62
:10CBD0000600A310019336D06C6A002C07D11020F8
:10CBE000FDF786FC6862446084600460C4606F6A1C
:10CBF000BC68002C07D116492800FFF740FF00232E
:10CC00000400B86003600122019B13420AD0310086
:10CC100022002800FFF73CFF070031002800FFF743
:10CC20008EFE3E00019B5B1001930CD02068002813
:10CC300007D1220021002800FFF72AFF00232060EF
:10CC400003600400DFE73000FEBDC04610E60000D0
:10CC500071020000F0B50D0017002B69541185B06A
:10CC6000E3180193013300934968AB680290009A7E
:10CC7000934235DB0298FFF72AFE002302000600EC
:10CC800019001432A3422EDBE343DB171C402B00B8
:10CC9000A40014192A69143392009A1894461F228A
:10CCA000174024D00132D21B0392002219682000C1
:10CCB000B9400A4304C404CB0399CA409C45F5D843
:10CCC0004260002A02D0019B02330093009B02982D
:10CCD000013B33612900FFF732FE300005B0F0BDA3
:10CCE00001315B00C3E7980011500133CAE704CB60
:10CCF00004C49C45FBD8E9E70A69036930B59B1A6F
:10CD00000DD192001430143184188918043C043970
:10CD100025680A68954204D00123954204D318007F
:10CD200030BDA042F2D3FAE75B42F8E7F0B50D0060
:10CD300085B00700110028001400FFF7DDFF061E74
:10CD400008D101003800FFF7C2FD012346610361ED
:10CD500005B0F0BD01230193002804DB23002C0063
:10CD60001D000023019361683800FFF7B0FD2F001C
:10CD70000022019B2669C3601434B300E3180293B8
:10CD80002B6914379B00FB1803930300944614335C
:10CD900020CC04CF0192AAB294446A46614692889C
:10CDA0002D0C8A1A0199090C691A151449190D14C8
:10CDB00092B209040A431A60039AAC460433BA4299
:10CDC000E6D802991A008C4205D3043A1368002B66
:10CDD0000ED00661BCE704CC91B261440D14120C74
:10CDE0005219151489B212040A43AC4604C3E8E789
:10CDF000013EEAE7F7B51D0001211400089FFFF787
:10CE000066FD2B036D0006001B0B6D0D24D10193F5
:10CE1000002C27D068460094FFF702FE009C0028F3
:10CE20001ED0019B20211A00091A8A40C3402243C8
:10CE300072610193019CB461631E9C4101343461B1
:10CE4000002D18D0124BED1835232D183D60181AFF
:10CE5000099B18603000FEBD802252031343D6E7C1
:10CE60007461E7E701A8FFF7DBFD0124019B346152
:10CE700073612030E4E7074BC018074B3860E318B4
:10CE80009B00F3185869FFF7B1FD6401201ADFE732
:10CE9000CDFBFFFFCEFBFFFFFFFFFF3F4A4370B517
:10CEA00011001400FDF73EFE051E03D022000021F4
:10CEB000FDF760FB280070BDF8B507000D001600F7
:10CEC000002905D11100FDF72DFE04002000F8BD5A
:10CED000002A03D1FDF7DCFD3400F7E700F046FA45
:10CEE0002C00B042F2D231003800FDF71BFE041EC8
:10CEF000ECD029003200FDF721FB29003800FDF7B6
:10CF0000C7FDE3E7F0B58E6885B007000C0003921B
:10CF100001939E423CD890238A89DB001A4234D088
:10CF20000325096923685B1A0293636902985D43CC
:10CF3000EB0F5D19019B6D1001331B18AB4200D93B
:10CF40001D00530532D529003800FDF7EBFD061E04
:10CF500009D10C233B6040230120A28940421343A6
:10CF6000A38105B0F0BD029A2169FDF7E7FAA38914
:10CF7000144A1A4080231343A381029B2661F618AA
:10CF800026606561019EED1AA560019B9E4200D955
:10CF9000019E320003992068FDF7D9FAA3680020AA
:10CFA0009B1BA36023689E192660DAE72A003800DD
:10CFB000FFF782FF061EE0D121693800FDF768FD0A
:10CFC000C7E7C0467FFBFFFFF0B59FB00290059317
:10CFD0008B890F0016001B0611D50B69002B0ED193
:10CFE0004021FDF79FFD38603861002805D10C23F2
:10CFF000029A013813601FB0F0BD40237B6100230B
:10D0000006AC6361203363761033A37635002B784A
:10D01000002B01D0252B46D1AB1B04930CD0320042
:10D0200039000298FFF76EFF431C00D1AEE0626941
:10D03000049B9446634463612B78002B00D1A5E0E8
:10D04000012200235242626002A9543252186E1C1F
:10D050002360E360A3601370A36531780522544810
:10D06000FFF728FC751C00281FD12268D30604D5C1
:10D07000532302A95B1820211970130704D55323E9
:10D0800002A95B182B21197033782A2B16D0350092
:10D0900000210A20E3682A786E1C303A092A4ED90A
:10D0A000002918D010E00135B1E7414B2268C01AC1
:10D0B00001238340134323602E00CEE7059B191DF7
:10D0C0001B680591002B01DB099304E05B42E360E0
:10D0D0000223134323602B782E2B0AD16B782A2B43
:10D0E00035D1059B02351A1D1B680592002B2BDBE1
:10D0F0000793304E297803223000FFF7DBFB00282E
:10D1000006D04023801B83402268013513432360EF
:10D110002978062228486E1C2176FFF7CBFB0028D1
:10D120003CD0264B002B25D10722059B0733934388
:10D13000083305936369039A9B18636166E7434369
:10D1400001219B183500A6E701235B42D0E70023AD
:10D150000A201A000135636029786E1C30390929CC
:10D1600003D9002BC5D00792C3E7424301235218CD
:10D170003500F1E705AB00933A00114B210002980E
:10D18000FDF7CAFD0390039B0133D3D1BB890B98F4
:10D190005B0600D42FE7012040422CE705AB00934B
:10D1A0003A00074B21000298FEF770F8EAE7C04604
:10D1B0001CE6000022E6000026E6000019AD000093
:10D1C00005CF00000EB4812370B59DB002AC21AD37
:10D1D0009B0040CDA38102900690FEF7ADF90B4B6A
:10D1E000606063620023606109486363A364013B7C
:10D1F000E38132002B0021000068019500F01AF94C
:10D200001DB070BC08BC03B01847C04615D2000062
:10D210003400002000207047F0B51F000E0085B0DC
:10D220000390019102920A983478FDF74FF9082291
:10D2300000194378751C134038D12D2C38D17478DF
:10D24000B51C01330093002F65D0102F09D1302C6D
:10D2500007D120222B789343582B57D110276C7875
:10D260000235012039004042FBF78EF9060001200B
:10D2700039004042FBF70EFA002301228C461800C9
:10D28000524221003039092917D80C00A74222DD6B
:10D29000002B1EDB1300864205D301D1A44502DB1F
:10D2A0000123784320182C780135EAE72E00BAE7ED
:10D2B0002B2CC7D1B51C7478C4E72100413919293A
:10D2C00001D8373CE2E721006139192903D8573CDE
:10D2D000DCE71300E7E7002B09DA22230120039A99
:10D2E00040421360029B002B0AD105B0F0BD009AAA
:10D2F000002A00D04042029A002AF6D0002B01D02A
:10D300006B1E0193029B019A1A60EEE73024002FF6
:10D31000A7D10827A5E7302C9BD00A27A1E700005A
:10D3200013B5054C2468246A002C00D1034C0094EA
:10D33000FFF772FF16BDC0463400002098000020A1
:10D3400037B51300064A05001068046A002C00D1A6
:10D35000044C0A0000942900FFF75EFF3EBDC04662
:10D360003400002098000020704770470B1F1B6896
:10D37000181F002B01DA0B58C018704770B5140045
:10D380004B1C03D101256D42280070BD93892022DA
:10D390009343626BA381CEB2CDB26368002A10D0F2
:10D3A000A26B9A4207DD2368013B23601E7063680D
:10D3B00001336360E8E7210000F052FB0028F2D05F
:10D3C000E0E721692268002907D0914205D2511E69
:10D3D0000878A84201D12160EAE72364230044339E
:10D3E00063630323A36323004633E2631E70236059
:10D3F0000123DEE710B50C00496B00290ED0230095
:10D400004433994201D0FDF743FB0020236C606355
:10D410006360834202D0E36B236010BD2369012067
:10D4200023600023A289636020331343A381404219
:10D43000F3E70000F0B5B94CC025A54405930023DF
:10D440000C004A934B93862107AB4C93BE2301906B
:10D45000170004A8B24A490040185B00C250B14A04
:10D460006D0042513B78002B00D154E1FDF732F8BA
:10D4700008223B787E1CC01802934378134023D0C7
:10D480006368002B14DDFDF725F8082123681A785E
:10D49000801842780A4201D13700E3E74B9A013302
:10D4A000029201324B9262682360013A6260E7E7C0
:10D4B000862204AB52009B185B592100019802930D
:10D4C00098470028DFD0E7E7029A252A6DD14993D3
:10D4D00047937B782A2B02D11A3B4793BE1C370017
:10D4E0000A2239787B1C03930B00303B092B24D98B
:10D4F0008D4E03223000FFF7DDF9002807D001230D
:10D50000801B8340479A039F1343049247933B78C1
:10D510007E1C672B35D8652B00D3BBE0472B14D876
:10D52000452B00D3B6E0002B00D1F1E0252B3CD0F9
:10D5300003234D930733489369E0499B039F04936A
:10D540005343303B59184991CBE75B2B00D17DE029
:10D5500010D8582BECD1479A02928022029992005F
:10D560000A434792102248926E229A429B415B42A4
:10D5700003334BE0632B00D175E0642BD8D10A2232
:10D58000F1E7702B38D008D86E2B00D173E03AD871
:10D59000692BCDD100234893EAE7752BEFD0782B88
:10D5A000D9D0732BC4D1022330E06368002B0FDD88
:10D5B000236802991A788A4200D0ACE0013362688D
:10D5C00023604B9B013A0293013362604B9363E704
:10D5D000862204AB52009B185B59210001980393EB
:10D5E00098470028E4D04A98002800D08CE0013801
:10D5F000A9239B009D44F0BD479A029220220299E4
:10D600000A434792A7E708234893043B4D93636876
:10D61000002B41DD479B02935B0608D4FCF75AFFC1
:10D62000082123681A78801842780A4240D14D9B1D
:10D63000022B55DC05AB220047A9019800F078F8D1
:10D64000012868D0022800D026E7CCE7310007A8DF
:10D6500000F0D6F9479B060002934023029A134339
:10D6600047930123D2E7479B02934023029A134337
:10D6700047930023CAE74798C30600D50CE7059BEC
:10D680004B9A191D05911B68C70701D51A8003E73E
:10D690001A6001E70523B9E7862204AB52009B1804
:10D6A0005B5921000198029398470028B2D09AE76D
:10D6B0004B9A029201324B926268013A6260002AF0
:10D6C00002DD01332360A9E7862204AB52009B18D8
:10D6D0005B59210001980293984700289ED082E769
:10D6E000042B06DC05AB220047A9019800F086F860
:10D6F000A6E70E4B002B00D1CEE605AB220047A9D2
:10D70000019800E000BF9BE7A3895B0600D46FE7A8
:10D71000012040426CE74A986AE7C0465CFDFFFF83
:10D720007DD30000F5D3000022E6000000000000D9
:10D73000F7B515008A6801900C00002A04D18A69A7
:10D74000002A17D10132A2602268D20603D41A68D7
:10D75000111D196017680026A369002B1FD0012B2B
:10D760000BD12B6862691B78D35C002B17D1002E7C
:10D7700033D109E001225242E5E7022B06D0002E08
:10D780002BD1A369012B28D10120FEBDFCF7A2FEFD
:10D7900008222B681B78C01843781342EFD110225F
:10D7A00023680136134203D12B681B783B70013785
:10D7B0002A686B6801322A60A268013B013A6B60FB
:10D7C000A260002A09D0002BC6DCC0235B00E3580E
:10D7D0002900019898470028BED0102322681340E2
:10D7E00006D1E2680132E260A269002A00D03B70F3
:10D7F000236900209E192661C7E70000F0B50C00E0
:10D800008BB00293784B0490160007AA23CB23C257
:10D81000764B0593A369032B01D1754B0593AE227B
:10D820000020A3685200591E0390914205D95E3B27
:10D83000FF3B03935E23FF33A36023001C3301935C
:10D84000D023002722681B0113432360019B009310
:10D85000336807A81978BB0002221858FFF72AF886
:10D8600000282BD0012F62D16368002B06D108332A
:10D8700022686360F933FF33134323605D4B2268F2
:10D8800013402360A3685A1EA260002B16D0336891
:10D890005A1C32601B78009A13707368551C013B48
:10D8A0007360002B09DCC0235B00E358310004984F
:10D8B00000939847002800D080E000950137032F9F
:10D8C000C6D16368002B01D10A33636010210027A1
:10D8D00063686069C91A484BC91800F091F8009D47
:10D8E000A36822680093002B41D0316863690878EF
:10D8F0001B5C002B3BD0302829D180231B011A420E
:10D9000025D0039B0137002B05D01A00009B013A5C
:10D9100001330392A3607368013B7360002B1DDD2C
:10D92000336801333360A368013BA360D8E7022F5B
:10D93000A8D1C02180232268C90011409B009942D0
:10D94000BFD1F13BFF3B6360F033134399E72B4BAF
:10D95000134023600B782B700135DCE7C0235B009C
:10D96000E35831000498009398470028DBD02368DF
:10D97000DB050ED5019B9D4207D9BE23013D5B000F
:10D980002978E358320004989847019B01209D4272
:10D9900027D0102223681A401CD12A70636801998D
:10D9A0000498059EB047029B21681B688A0607D52C
:10D9B0001A1D02990A601B68186008E00027D6E764
:10D9C0001A1DCE07F5D502990A601B681880E36816
:10D9D0000133E3600020019BED1A2369EF19DF1981
:10D9E00027610BB0F0BDC04630E6000021D3000037
:10D9F0006DB60000FFFAFFFF3CE60000FFF6FFFFF8
:10DA000070B50B7805005E2B18D04A1C0021280049
:10DA10006C1CFF3401700130A042FBD1501E002B62
:10DA20000BD001204140E9541478501C2D2C0CD00F
:10DA30005D2C02D0002C05D1100070BD8A1C4B78E3
:10DA40000121E4E723000200EDE756785D2EF9D0CE
:10DA5000B342F7DC02320133E9549E42FBDCE3E7D8
:10DA60000B00F7B54D6B44330C009D421CD1802652
:10DA7000F6003100FDF756F8002802D1012040429F
:10DA8000FEBD23006063A66346331A78104BC25470
:10DA9000230045331A780F4BC2542A780E4BC254D8
:10DAA000C01820600020EBE78E6B290073001A007D
:10DAB0000193FFF701FA051EE0D08719010032003B
:10DAC0003800FCF73BFD019B27606563A363E9E732
:10DAD000FF030000FE030000FD030000044A13687A
:10DAE000002B00D1034B1818106018007047C04677
:10DAF0001C1000200C110020F8B5C046F8BC08BC72
:10DB00009E467047F8B5C046F8BC08BC9E467047B4
:10DB1000436C6F736520426C696E6420456E6420AF
:10DB2000506F736974696F6E3A2000417474656D4B
:10DB30007074696E6720746F20636F6E6E656374B6
:10DB400020746F20535349443A20002E00596F75BA
:10DB500027726520636F6E6E656374656420746FF1
:10DB600020746865206E6574776F726B004F706506
:10DB70006E20426C696E6420456E6420506F73693C
:10DB800074696F6E3A2000787377325853574000AB
:10DB9000446173576966690025004E6F772066728D
:10DBA0006F6D2054696D654C6962206D6F64756C92
:10DBB000653A20003A002F004E6F772066726F6D35
:10DBC000207468652057694669206D6F64756C65BF
:10DBD0003A20001F1C1F1E1F1E1F1F1E1F1E1F7707
:10DBE0006966693130312D252E3258252E32580084
:10DBF00077696669313031000000000000000000E4
:10DC0000F12F00002D310000ED2F00002330000027
:10DC10005130000005300000993000001D32000036
:10DC2000813200006930000035300000BD30000056
:10DC300025300000D5300000FD3000000020C3C9B1
:10DC4000C4CA0009121B242D363F48415A536C6543
:10DC50007E7719100B023D342F265158434A757CAC
:10DC6000676E323B2029161F040D7A7368615E5778
:10DC70004C452B2239300F061D14636A7178474ECC
:10DC8000555C646D767F4049525B2C253E37080118
:10DC90001A137D746F6659504B42353C272E11186C
:10DCA000030A565F444D727B60691E170C053A33B8
:10DCB00028214F465D546B627970070E151C232A8C
:10DCC00031384148535A656C777E09001B122D2468
:10DCD0003F3658514A437C756E671019020B343D2C
:10DCE000262F737A6168575E454C3B3229201F16F8
:10DCF0000D046A6378714E475C55222B3039060F4C
:10DD0000141D252C373E0108131A6D647F76494097
:10DD10005B523C352E2718110A03747D666F5059EB
:10DD2000424B171E050C333A21285F564D447B7237
:10DD300069600E071C152A233831464F545D626B0B
:10DD40007079000000000000000000002552000073
:10DD50002752000001020300000000000000000044
:10DD60001D570000915700002F5700003957000041
:10DD7000FD5600009D570000E15700001D590000AE
:10DD80001D5800001B5700001B570000CD58000015
:10DD90001F570000000000001600000008000000EF
:10DDA0001C000000FF00000400040600000000004A
:10DDB00017000000080000001C000000FF00010424
:10DDC00001040700000000000A0000000800000035
:10DDD0001C000000120000010001FF000000000014
:10DDE0000B000000080000001C00000013000101EF
:10DDF0000101FF00010000000A000000080000000F
:10DE00001C000000FF00000500050A0001000000E2
:10DE10000B000000080000001C000000FF000105CE
:10DE200001050B00000000001400000008000000C5
:10DE30002C000000FF0002000200040000000000AF
:10DE400015000000080000002C000000FF00030087
:10DE500003000500000000001000000002000000A8
:10DE60001C000000FF000002000200000000000093
:10DE7000110000000200000004000000FF00FFFF8E
:10DE8000FFFF01000000000013000000020000007E
:10DE90001C000000FF0001030103FF000000000060
:10DEA00008000000030000001C000000100000003B
:10DEB0000000100000000000090000000300000046
:10DEC000040000001100FFFFFFFFFF000100000041
:10DED000170000000300000004000000FF00FFFF27
:10DEE000FFFFFF000100000016000000030000001B
:10DEF00004000000FF00FFFFFFFFFF000000000024
:10DF00000200000001000000060000000000FFFF0A
:10DF1000FFFFFF0001000000020000000100000000
:10DF2000040000000A00FFFFFFFF020001000000E4
:10DF30000300000001000000040000000B00FFFFD0
:10DF4000FFFF0300000000000400000001000000CB
:10DF50001C000000040000000000FF0000000000A2
:10DF600005000000010000001C0000000500010089
:10DF70000100FF000000000006000000010000009A
:10DF8000040000000600FFFFFFFFFF00000000008C
:10DF90000700000001000000040000000700FFFF70
:10DFA000FFFFFF0000000000180000000600000056
:10DFB00000000000FF00FFFFFFFFFF000000000067
:10DFC000190000000600000000000000FF00FFFF35
:10DFD000FFFFFF000000000012000000080000002A
:10DFE00004000000FF00FFFFFFFFFF000000000033
:10DFF000030000000800000004000000FF00FFFF15
:10E00000FFFFFF00000000000C0000000300000004
:10E0100000000000FF00FFFFFFFFFF000000000006
:10E020000D0000000300000000000000FF00FFFFE3
:10E03000FFFFFF00000000000E00000008000000CD
:10E0400000000000FF00FFFFFFFFFF0000000000D6
:10E050000F0000000300000000000000FF00FFFFB1
:10E06000FFFFFF00000000001B0000000800000090
:10E0700000000000FF00FFFFFFFFFF0000000000A6
:10E080001C0000000800000000000000FF00FFFF6F
:10E09000FFFFFF0001000000080000000800000072
:10E0A00000000000FF00FFFFFFFFFF000100000075
:10E0B000090000000800000000000000FF00FFFF52
:10E0C000FFFF090000000000000000000800000041
:10E0D00000000000FF00FFFFFFFFFF000000000046
:10E0E000010000000800000000000000FF00FFFF2A
:10E0F000FFFFFF0000000000000000002967000093
:10E10000616900002567000045690000256900007D
:10E110009D690000816900002167000023670000FD
:10E1200011690000C1690000536900003D670000EB
:10E13000A366000069680000CD660000F0FFFFFFE5
:10E14000000000000169000059680000E969000052
:10E150001167000000000000000000001D6C0000BE
:10E1600023780000FB77000007780000856A000034
:10E17000876A0000756B000041726475696E6F20DC
:10E180004D4B523130303000040309044172647544
:10E19000696E6F204C4C430012010002EF020140F7
:10E1A00041234E8000010102030100000000000035
:10E1B00000000000817D0000758000000B7A0000E7
:10E1C000577A0000057A00001D7E00001B7A0000CF
:10E1D000F5790000B57A0000337A0000F17900008B
:10E1E0000000000000000000677E00000D0A00250E
:10E1F0002525642E25646600CC9100003E90000029
:10E2000082900000E68F0000829000007291000072
:10E2100082900000E68F00003E9000003E900000DB
:10E2200072910000E68F0000DE8F0000DE8F00009C
:10E23000DE8F000080910000F4980000F697000047
:10E24000F6970000149B0000F0970000F097000084
:10E25000FC9A0000149B0000F0970000FC9A00005C
:10E26000F0970000149B00000A9B00000A9B00002E
:10E270000A9B0000189B00004300504F5349580070
:10E280001F0000001C0000001F0000001E00000016
:10E290001F0000001E0000001F0000001F00000003
:10E2A0001E0000001F0000001E0000001F000000F4
:10E2B000000000001F0000003B0000005A000000AA
:10E2C0007800000097000000B5000000D4000000B6
:10E2D000F300000011010000300100004E010000B9
:10E2E000494E4600696E66004E414E006E616E00FA
:10E2F000303132333435363738394142434445467C
:10E300000030313233343536373839616263646511
:10E310006600545A00474D54002531305B5E302D65
:10E32000392C2B2D5D256E004D256875256E2E250B
:10E330006875256E2E256875256E002F2568752554
:10E340006E3A256875256E3A256875256E000020A1
:10E350002020202020202020282828282820202095
:10E360002020202020202020202020202020208845
:10E3700010101010101010101010101010101004A9
:10E3800004040404040404040410101010101010F9
:10E3900041414141414101010101010101010101ED
:10E3A0000101010101010101010110101010101003
:10E3B00042424242424202020202020202020202BD
:10E3C00002020202020202020202101010102000D9
:10E3D000000000000000000000000000000000003D
:10E3E000000000000000000000000000000000002D
:10E3F000000000000000000000000000000000001D
:10E40000000000000000000000000000000000000C
:10E4100000000000000000000000000000000000FC
:10E4200000000000000000000000000000000000EC
:10E4300000000000000000000000000000000000DC
:10E440000000000000000000000000000000004983
:10E450006E66696E697479004E614E0000000000BE
:10E4600000000000000000000000000000000000AC
:10E47000000000000000000000000000000000009C
:10E48000000000000000000000000000000000008C
:10E49000000000000000000000000000000000007C
:10E4A000000000000000000000000000000000006C
:10E4B0000000000000000000000000001F0000003D
:10E4C0001C0000001F0000001E0000001F000000D4
:10E4D0001E0000001F0000001F0000001E000000C2
:10E4E0001F0000001E0000001F0000001F000000B1
:10E4F0001D0000001F0000001E0000001F000000A3
:10E500001E0000001F0000001F0000001E00000091
:10E510001F0000001E0000001F000000000000009F
:10E520000080E03779C34143176E05B5B5B893460F
:10E53000F5F93FE9034F384D321D30F94877825ADB
:10E540003CBF737FDD4F1575000000000000F03FF9
:10E5500000000000000024400000000000005940BE
:10E560000000000000408F40000000000088C34011
:10E5700000000000006AF8400000000080842E4186
:10E5800000000000D01263410000000084D79741D2
:10E590000000000065CDCD41000000205FA00242D8
:10E5A000000000E876483742000000A2941A6D424D
:10E5B000000040E59C30A2420000901EC4BCD64240
:10E5C00000003426F56B0C430080E03779C34143EB
:10E5D00000A0D8855734764300C84E676DC1AB4361
:10E5E000003D9160E458E143408CB5781DAF15447F
:10E5F00050EFE2D6E41A4B4492D54D06CFF080445A
:10E60000F64AE1C7022DB544B49DD9794378EA446E
:10E6100005000000190000007D000000232D302BB4
:10E620002000686C4C0065666745464700000000A6
:10E630004EE6000051E6000054E60000412D466120
:10E640002D66383930313233343536375D002B2D75
:0CE650000030300078580000000000008E
:10E65C00000000000F0000002C0100001F1C211EF8
:10E66C000001000040420F000A0000000A000000F8
:10E67C00FFFFFFFFFFFFFFFF00C2010000000800CB
:10E68C00FFFFFFFF38000020000000007CE40000CA
:10E69C009CE400005CE400000000000000000000AE
:10E6AC00000000000000000000000000000000005E
:10E6BC00000000000000000000000000000000004E
:10E6CC00000000000000000000000000000000003E
:10E6DC00000000000000000000000000000000002E
:10E6EC0000000000000000004300000000000000DB
:10E6FC00000000000000000000000000000000000E
:10E70C0000000000000000004300000000000000BA
:10E71C0000000000000000000000000000000000ED
:10E72C00000000000000000043000000000000009A
:10E73C0000000000000000000000000000000000CD
:10E74C00000000000000000043000000000000007A
:10E75C0000000000000000000000000000000000AD
:10E76C00000000000000000043000000000000005A
:10E77C00000000000000000000000000000000008D
:10E78C00000000000000000043000000000000003A
:10E79C00000000000000000000000000000000006D
:10E7AC00000000000000000043000000000000001A
:10E7BC00000000000000000000000000000000004D
:10E7CC000000000000000000FDBA000019A50000C8
:10E7DC00000000004EE300004BDB0000EEE1000007
:10E7EC00EEE10000EEE10000EEE10000EEE10000E1
:10E7FC00EEE10000EEE10000EEE10000EEE10000D1
:10E80C00FFFFFFFFFFFFFFFFFFFFFFFFFFFF00000A
:10E81C000100415343494900000000000000000082
:10E82C0000000000000000000000000000000000DC
:10E83C000000415343494900000000000000000063
:10E84C0000000000000000000000000000000000BC
:10E85C000000000015E3000015E3000000000000BC
:10E86C0001000000000000004A0000000000000051
:10E87C00000000000000000000000000000000008C
:10E88C00000000000000000000000000000000007C
:10E89C004A00000000000000000000000000000022
:10E8AC00000000000000000000000000000000005C
:10E8BC00000000000000000018100020DD20000007
:10E8CC000D240000C92F00009D330000D956000014
:10E8DC0055590000FD590000716A00008578000050
:10E8EC00557F0000B5200000000000000000000073
:0400000300005C7528
:00000001FF
